S0120000426F6F746C6F616465722E7372656307
S315019F0000FFFFFFFFFFFFFFFFFFFFFFFFFFFFFFFF5A
S315019F0010FFFFFFFFFFFFFFFFFFFFFFFFFFFFFFFF4A
S315019F0020FFFFFFFFFFFFFFFFFFFFFFFFFFFFFFFF3A
S315019F0030FFFFFFFFFFFFFFFFFFFFFFFFFFFFFFFF2A
S315019F0040FFFFFFFFFFFFFFFFFFFFFFFFFFFFFFFF1A
S315019F0050FFFFFFFFFFFFFFFFFFFFFFFFFFFFFFFF0A
S315019F0060FFFFFFFFFFFFFFFFFFFFFFFFFFFFFFFFFA
S315019F0070FFFFFFFFFFFFFFFFFFFFFFFFFFFFFFFFEA
S315019F0080FFFFFFFFFFFFFFFF3412F759FFFFFFFF40
S315019F0090FFFFFFFFFFFFFFFFFFFFFFFFFFFFFFFFCA
S315019F00A0FFFFFFFFFFFFFFFFFFFFFFFFFFFFFFFFBA
S315019F00B0FFFFFFFFFFFFFFFFFFFFFFFFFFFFFFFFAA
S315019F00C0FFFFFFFFFFFFFFFFFFFFFFFFFFFFFFFF9A
S315019F00D0FFFFFFFFFFFFFFFFFFFFFFFFFFFFFFFF8A
S315019F00E0FFFFFFFFFFFFFFFF74A0A001FFFFFFFFC1
S315019F00F07B3A2D29FFFFFFFFFFFFFFFFFFFFFFFF5B
S315019F0100FFFFFFFFFFFFFFFF3CFFFFFFFFFFFFFF1C
S315019F011055FFFFFFFFFFFFFF00000000FFFFFFFFEF
S315019F012000000001FFFFFFFF00000000FFFFFFFF30
S315019F013000000080FFFFFFFF0000FFFFFFFFFFFFA3
S315019F0140FFFDFFFFFFFFFFFF7B3A2D29FFFFFFFF0C
S31501A0000004F01FE574A0A001DFF8A41808707047DA
S31501A00010DFF8A008006880098001DFF89818086059
S31501A00020DFF894080078C0B20028F9D10120DFF8E2
S31501A000308C18087070472DE9F14F82B00298006BB9
S31501A00040DFF87C1808600298406BDFF87818086022
S31501A000500298806BDFF870180860002006004FF444
S31501A00060D27060F30E06012060F31D7601F006E85A
S31501A0007072B626F04046DFF854180E60012161F3EE
S31501A000809F76DFF848180E60022161F39F76DFF8AC
S31501A000903C180E6056F04046DFF830180E6000217D
S31501A000A0DFF82C28118000F0EEEF0121DFF82428DB
S31501A000B01170DFF820080078C0B20028F9D001201D
S31501A000C0DFF814180870FFF7A3FF0020DFF80C185B
S31501A000D008700020DFF8081808700020DFF804185F
S31501A000E008700020DFF8001808700020DFF8FC1760
S31501A000F008700020DFF8F81708700020DFF8F41761
S31501A0010008700020DFF8F01708700020DFF8EC1760
S31501A0011008700120DFF8E817096860F31841DFF8D5
S31501A00120E00701600120DFF8DC17096860F31441DC
S31501A00130DFF8D00701600B20DFF8CC1708700B2081
S31501A00140DFF8C017096860F30C21DFF8B807016072
S31501A001500220DFF8AC17096860F30601DFF8A007F3
S31501A0016001600220DFF89C17096860F30711DFF828
S31501A00170940701600220DFF88817096860F35F61C0
S31501A00180DFF87C0701600220DFF87817096860F3C1
S31501A001900301DFF870070160DFF870070700002090
S31501A001A083461FFA8BFBBBF5885F05D2002038601A
S31501A001B03F1D1BF1010BF4E7002080460020ADF89E
S31501A001C00000DFF84C0700686FF38F00DFF84017D7
S31501A001D008608020DFF83C17096860F38F01DFF81B
S31501A001E03407016002988246002083461FFA8BFBE2
S31501A001F0BBF1030F44D29AF8000001283BD1DAF8EB
S31501A002000400002837D0002081464846BAF80210DB
S31501A0021080B288422FD2DFF8F406DFF8F416096817
S31501A00220C1F38D0100EB81001FFA88F800EB88006D
S31501A0023004000220216860F39F712160206850F0BC
S31501A0024060502060DAF804001FFA89F950F82900F5
S31501A00250216860F31A412160BDF800001FFA88F8F1
S31501A0026018FA80F0216860F30A01216018F10108EB
S31501A0027019F10109C9E71AF1080A1BF1010BB5E742
S31501A00280ADF8008002988246002083461FFA8BFBB8
S31501A00290BBF1030F33D29AF8000002282AD1DAF86B
S31501A002A00400002826D0DFF86406DFF86416096882
S31501A002B0C1F38D0100EB81001FFA88F800EB8800DD
S31501A002C00400206820F0404020600120216860F3EE
S31501A002D0DD612160DAF804000068216860F31A4143
S31501A002E02160DAF804004068216860F30A01216000
S31501A002F018F101081AF1080A1BF1010BC6E7DFF88C
S31501A003008C0C80F800800020804602981830824626
S31501A00310002083461FFA8BFBBBF1030F44D29AF848
S31501A00320000001283BD1DAF80400002837D00020CC
S31501A0033081464846BAF8021080B288422FD2DFF829
S31501A00340CC05DFF8D0150968C1F38D0100EB81005A
S31501A003501FFA88F800EBC80005000220696860F35F
S31501A003609F716960286850F060402860DAF804003F
S31501A003701FFA89F950F82900296860F31C01296040
S31501A00380BDF800001FFA88F818FA80F0696860F3D2
S31501A003901C01696018F1010819F10109C9E71AF1EF
S31501A003A0080A1BF1010BB5E7BDF8000018EB000028
S31501A003B0DFF8DC1B087002981830824600208346BD
S31501A003C01FFA8BFBBBF1030F33D29AF80000022868
S31501A003D02AD1DAF80400002826D0DFF83005DFF8A4
S31501A003E034150968C1F38D0100EB81001FFA88F865
S31501A003F000EBC8000500686820F040406860012055
S31501A00400296860F35F712960DAF804000068296839
S31501A0041060F31C012960DAF804004068696860F39A
S31501A004201C01696018F101081AF1080A1BF1010BF8
S31501A00430C6E71FFA88F8DFF8DC04006868F31640FF
S31501A00440DFF8D01408600120DFF8481B096860F3C3
S31501A004500511DFF8400B01600220DFF8381B09689F
S31501A0046060F38301DFF82C0B01600120DFF8281B64
S31501A0047008700120DFF8241B0870DFF8240B006840
S31501A0048070F06040DFF8181B08600020DFF8141B2D
S31501A004900870DFF8140B006830F0FE40DFF8081B87
S31501A004A008601020DFF8001B096860F31641DFF829
S31501A004B0F80A01604FF48070DFF8EC1A096860F35E
S31501A004C08F01DFF8E40A01600020DFF8E01A087066
S31501A004D0DFF8DC0A006830F0FE40DFF8D41A0860C5
S31501A004E01020DFF8CC1A096860F31641DFF8C00ABC
S31501A004F001604FF4B060DFF8B81A096860F38F01A4
S31501A00500DFF8AC0A01604FF42060DFF8A81A096889
S31501A0051060F38F01DFF89C0A0160DFF89C0A00688E
S31501A00520C008C000DFF8901A0860DFF88C0A0068DE
S31501A0053030F07000DFF8801A0860DFF87C0A0068E6
S31501A0054030F4E060DFF8701A0860DFF8700A00681E
S31501A0055030F07C50DFF8641A0860DFF8600A0068A2
S31501A0056030F47C10DFF8541A08604FF46860DFF8A5
S31501A005704C1A096860F38F01DFF8400A0160002078
S31501A00580DFF83C1A0870DFF83C0A006830F07C50AE
S31501A00590DFF8301A08602020DFF8281A096860F30E
S31501A005A01541DFF8200A01604FF46C60DFF8141AD8
S31501A005B0096860F38F01DFF80C0A0160DFF8080A09
S31501A005C00068C008C000DFF8001A08600020DFF844
S31501A005D0FC1908600020DFF8F81908600020DFF890
S31501A005E0F41908607FF04040DFF8EC19086000209C
S31501A005F0DFF8E81908600120DFF8E4190870012086
S31501A00600DFF8E01908700120DFF8DC190870012075
S31501A00610DFF8D81908700120DFF8D4190870012075
S31501A00620DFF8D01908700020DFF8CC190870002077
S31501A00630DFF8C81908700120DFF8C4190870002076
S31501A00640DFF8C01908700020A2490870A1480078F7
S31501A00650C0B20028FAD10020DFF8AC190860BDE8C5
S31501A00660F78F80B51F220FF2B021282000F08AFD56
S31501A0067001BD2DE9F84F04000D0016001F00F6B2CA
S31501A00680002E04D0F6B2092E01D2002F0BD18D482F
S31501A006900068002800F0B8800121ADB22800894A7F
S31501A006A012689047B0E0DFF8640900788DF8000081
S31501A006B09DF8000000280BD082480068002800F0B1
S31501A006C0A3800121ADB228007E4A126890479BE023
S31501A006D0DFF8F80800680121A9400843DFF8EC1803
S31501A006E00860A9468948DFF8DC180968C1F38D01BD
S31501A006F000EB81001FFA89F95FEA091108448346D4
S31501A00700DBF8000050F08040CBF80000DBF80000D9
S31501A0071064F31C00CBF80000DBF8000020F00040D9
S31501A00720CBF80000DBF8000030F00050CBF8000059
S31501A00730DBF8040030F48000CBF80400DBF80400F9
S31501A0074030F0FF40CBF80400F6B2DBF8040066F304
S31501A007501340CBF80400DBF8040030F40010CBF80A
S31501A007600400DBF8040030F48010CBF80400F6B2E4
S31501A00770052E03D20020CBF80C001BE000208246F8
S31501A00780082080465FFA88F8B8F1050F10D3B8F1B2
S31501A0079001085FEA0A2A40463100C0B2C9B28842BE
S31501A007A0F0D25FFA88F817F8080050EA0A0AE9E7D2
S31501A007B0CBF80CA000208246042080465FFA88F878
S31501A007C0B8F1000F10D0B8F101085FEA0A2A404635
S31501A007D03100C0B2C9B28842F0D25FFA88F817F8E0
S31501A007E0080050EA0A0AE9E7CBF808A0012010FAA6
S31501A007F009F08246DFF81808C0F800A0DFF814084F
S31501A008000068DFF804180860BDE8F18FDFF8080872
S31501A008100078C0B2012803D10120DFF800180880B2
S31501A00820DFF8FC070078C0B2012807D10120DFF864
S31501A00830F01708700220DFF8E4170880DFF8E40754
S31501A008400078C0B2012807D10120DFF8D8170870B7
S31501A008500320DFF8C8170880DFF8CC070078C0B2FC
S31501A00860012807D10120DFF8C01708700420DFF89E
S31501A00870AC170880DFF8B4070078C0B2012807D109
S31501A008800120DFF8A81708700520DFF89017088067
S31501A00890DFF89C070078C0B2012807D10120DFF854
S31501A008A0901708700620DFF87417088070470000BB
S31501A008B0A2540000008C68B02060C4B00860C4B027
S31501A008C0B43A0000B83A0000BC3A0000009474B4EF
S31501A008D0A48174B4C000C0B4C100C0B4CE00C0B479
S31501A008E0C900C0B4C800C0B4C700C0B4C600C0B473
S31501A008F0C500C0B4C400C0B4C200C0B47700C0B4BF
S31501A009001C0090B40C0090B41D0090B4008090B46B
S31501A00910840090B4880090B404E04EE2FF5F2DE914
S31501A00920100AF1EE01002DE904D04DE2100B2DEDD8
S31501A0093010D04DE29C069FE5000090E5F0169FE5DC
S31501A00940000011E10000000AAFFFFFFAE4069FE5EF
S31501A009500000D0E57000EFE6000050E3D700000AE2
S31501A009600100A0E3CC169FE50000C1E50100A0E3CC
S31501A00970A4FDFFFAC0069FE5000090E5000050E344
S31501A009806400000AB0069FE5000090E500008DE531
S31501A009900000A0E30090B0E10000E0E30060B0E158
S31501A009A00000A0E30080B0E10800B0E17000EFE62E
S31501A009B0060050E31000002A8990B0E100009DE5F1
S31501A009C0000016E10000001A019099E26C069FE56D
S31501A009D00810B0E17110EFE60111B0E1010090E756
S31501A009E00910B0E17110FFE60111B0E1010090E735
S31501A009F00060B0E1018098E2EAFFFFEA40069FE5C8
S31501A00A00AC159FE5001091E55111EDE70111B0E19B
S31501A00A10010090E00910B0E17110FFE60112B0E10A
S31501A00A20010090E00070B0E1000097E5500FE0E70B
S31501A00A30000050E30300000A000097E5E004D0E3BC
S31501A00A400050B0E1030000EA000097E5E004D0E31E
S31501A00A504009B0E10050B0E1040097E52008B0E1FB
S31501A00A600F0010E20040B0E10400B0E17000EFE633
S31501A00A70090050E30100003A0800A0E30040B0E1FC
S31501A00A800000A0E300B0B0E10B00B0E10410B0E1BA
S31501A00A907000EFE67110EFE6010050E10F00002AA9
S31501A00AA003001BE30600001A0B00B0E17000EFE69D
S31501A00AB04001B0E10001B0E1000097E0080090E537
S31501A00AC000A0B0E104008DE20B10B0E17110EFE6D9
S31501A00AD001A0C0E72AA4B0E101B09BE2E9FFFFEAC9
S31501A00AE060059FE5000090E5000050E30600000ABE
S31501A00AF004208DE20410B0E17110EFE60500B0E12B
S31501A00B0040359FE5003093E533FF2FE128059FE5AA
S31501A00B10006080E596FFFFEA2C059FE5000090E5C1
S31501A00B20000050E36500000A1C059FE5000090E562
S31501A00B3000008DE50000A0E30090B0E10000E0E335
S31501A00B400060B0E10000A0E30080B0E10800B0E1E0
S31501A00B507000EFE6060050E31000002A8990B0E18C
S31501A00B6000009DE5000016E10000001A019099E23F
S31501A00B70C8049FE50810B0E17110EFE60111B0E1DC
S31501A00B80010090E70910B0E17110FFE60111B0E193
S31501A00B90010090E70060B0E1018098E2EAFFFFEA78
S31501A00BA0209099E298049FE504149FE5001091E531
S31501A00BB05111EDE70111B0E1010090E00910B0E19A
S31501A00BC07110FFE60112B0E1010090E00070B0E102
S31501A00BD0000097E5500FE0E7000050E30300000A8C
S31501A00BE0000097E5E004D0E30050B0E1030000EA7D
S31501A00BF0000097E5E004D0E34009B0E10050B0E180
S31501A00C00040097E52008B0E10F0010E20040B0E132
S31501A00C100400B0E17000EFE6090050E30100003ADC
S31501A00C200800A0E30040B0E10000A0E300B0B0E1FD
S31501A00C300B00B0E10410B0E17000EFE67110EFE631
S31501A00C40010050E10F00002A03001BE30600001A71
S31501A00C500B00B0E17000EFE64001B0E10001B0E1A8
S31501A00C60000097E0080090E500A0B0E104008DE245
S31501A00C700B10B0E17110EFE601A0C0E72AA4B0E124
S31501A00C8001B09BE2E9FFFFEAB8039FE5000090E50A
S31501A00C90000050E30600000A04208DE20410B0E132
S31501A00CA07110EFE60500B0E198339FE5003093E5BA
S31501A00CB033FF2FE190039FE5006080E595FFFFEAF2
S31501A00CC088039FE50000D0E57000EFE6000050E341
S31501A00CD05900000A0100A0E370139FE50000C1E5D9
S31501A00CE00100A0E3C7FCFFFA64039FE5000090E5BD
S31501A00CF07F0010E35000000A54039FE5000090E531
S31501A00D005004E5E70090B0E134039FE594129FE516
S31501A00D10001091E55111EDE70111B0E1010090E05C
S31501A00D200910B0E17110FFE60112B0E1010090E0F7
S31501A00D300070B0E1000097E5500FE0E7000050E336
S31501A00D400300000A000097E5E004D0E30050B0E1FB
S31501A00D50030000EA000097E5E004D0E34009B0E112
S31501A00D600050B0E1040097E52008B0E10F0010E2C1
S31501A00D700040B0E10400B0E17000EFE6090050E3E5
S31501A00D800100003A0800A0E30040B0E10000A0E3A2
S31501A00D9000B0B0E10B00B0E10410B0E17000EFE6E5
S31501A00DA07110EFE6010050E10F00002A03001BE3DA
S31501A00DB00600001A0B00B0E17000EFE64001B0E1B9
S31501A00DC00001B0E1000097E0080090E500A0B0E1C5
S31501A00DD004008DE20B10B0E17110EFE601A0C0E7AF
S31501A00DE02AA4B0E101B09BE2E9FFFFEA54029FE524
S31501A00DF0000090E5000050E30600000A04208DE201
S31501A00E000410B0E17110EFE60500B0E134329FE5C0
S31501A00E10003093E533FF2FE134029FE5000090E512
S31501A00E205004E5E72C129FE5001091E51010C5E7E7
S31501A00E3020029FE5001080E5AAFFFFEA18029FE5C0
S31501A00E400000D0E57000EFE6000050E31100000AB3
S31501A00E500100A0E300129FE50000C1E50100A0E3A7
S31501A00E6068FCFFFAF4019FE5000090E57F0010E31E
S31501A00E700800000AE4019FE5000090E55004E5E7BB
S31501A00E80DC119FE5001091E51010C5E7D0019FE5A3
S31501A00E90001080E5F2FFFFEAC8019FE50000D0E55A
S31501A00EA07000EFE6000050E30200000A0100A0E393
S31501A00EB0B0119FE50000C1E5AC019FE50000D0E5BA
S31501A00EC07000EFE6000050E31100000A40019FE523
S31501A00ED0000090E50060B0E1EC009FE5000090E520
S31501A00EE0066010E084019FE5000090E5000050E354
S31501A00EF00400000A0010A0E30600B0E16C219FE502
S31501A00F00002092E532FF2FE10100A0E358119FE5F1
S31501A00F100000C1E508019FE50000D0E57000EFE6FD
S31501A00F20000050E30200000A0100A0E3F0109FE5D3
S31501A00F300000C1E5E4009FE50000D0E57000EFE602
S31501A00F40000050E30200000A0100A0E3CC109FE5D7
S31501A00F500000C1E52800A0E314119FE5000081E58A
S31501A00F6010D08DE2100BBDEC04D08DE20100BDE8DE
S31501A00F70100AE1EEFF9FFDE824480078C0B20028E0
S31501A00F8002D000203C49087070470000860090B44A
S31501A00F90A3540000800090B40104C0B40004C0B4FE
S31501A00FA0900090B41F05C0B4A00090B49F05C0B432
S31501A00FB0B00090B4AC0090B4BC0090B4F00090B472
S31501A00FC01E06C0B4C00090B4C80090B4E00090B4AE
S31501A00FD0E40090B4540090B4500090B4580090B47A
S31501A00FE0B302C0B4A002C0B4A402C0B4BB02C0B4D0
S31501A00FF0BC02C0B4A902C0B4AA02C0B4B902C0B4AA
S31501A01000E002C0B4E102C0B4B03A00002702C0B405
S31501A01010D00090B4D80090B49D02C0B498540000FA
S31501A010209C02C0B49B02C0B49A02C0B49902C0B4D7
S31501A010309502C0B4EEE0F73F9302C0B4980090B415
S31501A010400CA7A001008090B4B43A00009C0090B413
S31501A010508002C0B4A40090B4A80090B48402C0B425
S31501A01060B40090B4B80090B48A02C0B48902C0B4E6
S31501A01070B83A0000480C40B0C000C0B400000FE16F
S31501A010801EFF2FE100C00FE1C0C0CCE3C00000E20B
S31501A0109000C08CE10CF021E11EFF2FE110B45949EB
S31501A010A0594A5A4B5A4C23605A4B1B78DBB2002B38
S31501A010B0FAD00023584C237000231800202805D20B
S31501A010C00FF26C1341F82030401CF7E700231800FB
S31501A010D0FF2805D80FF25C1342F82030401CF7E731
S31501A010E010BC704701204C4908704C48484908601B
S31501A010F0704770B4434C4A4D4A4E3678F6B2002E2C
S31501A011003ED180B220283BD2D2B2102A38D280B2A8
S31501A0111044F8201080B28608330080B210F003068E
S31501A01120002E05D0022E17D00CD3032E1ED027E0F9
S31501A01130D2B29BB255F8236062F303069BB245F87F
S31501A0114023601DE0D2B29BB255F8236062F30B2651
S31501A011509BB245F8236013E0D2B29BB255F8236047
S31501A0116062F313469BB245F8236009E0D2B29BB263
S31501A0117055F8236062F31B669BB245F82360FFE72F
S31501A0118070BC7047F0B4204C274D284E254F3F78B0
S31501A01190FFB2002F34D180B2FF2831D8D2B2202A93
S31501A011A02ED280B244F8201080B287083B009BB2B1
S31501A011B013F00307002F05D0022F0CD006D3032F5F
S31501A011C00ED012E09BB205F823200EE09BB205EBF0
S31501A011D083077A7009E09BB205EB8307BA7004E036
S31501A011E09BB205EB8307FA70FFE780B247093B0084
S31501A011F0012710F01F0C17FA0CF79BB246F82370C3
S31501A01200F0BC7047100040B0900040B011C9AC17B7
S31501A01210300D40B0780010B1C06410B1110CB117F7
S31501A01220900840B0D06410B1B00840B0800B40B077
S31501A01230FEFFFFEAFEFFFFEA80B500F04FFE00F0D9
S31501A01240A3FE00F06AFA00F0A7FD01BDDFF8301D8C
S31501A0125009884118DFF8282D11807047F8B50400D8
S31501A012600D001600DFF82C0B0078002804D0092108
S31501A01270200000F0F2F8EFE0B6B2002E02D0B6B22E
S31501A01280FB2E04D30921200000F0E7F8E4E0DFF803
S31501A01290480C0460DFF8400C868000200700380067
S31501A012A0C0B2310080B289B2884208D2FFB2E85DED
S31501A012B0DFF8241CFFB2394488717F1CEFE70020B8
S31501A012C0DFF8D01A4870DFF8CC0A8680FF20DFF855
S31501A012D0C41A88727F20DFF8BC1A0873DFF8B40A33
S31501A012E08088082843D20120DFF8A81AC880DFF831
S31501A012F0A40A8088DFF89C1A48800120DFF8941A96
S31501A013000881DFF8D40B0068DFF8701C0860DFF8ED
S31501A013106C0C007910F00F00DFF8601C0871DFF883
S31501A01320740A8088DFF8541C097960F30301DFF899
S31501A013304C0C0171DFF85C0A8088401CDFF83C1C6C
S31501A013400873002007003800C0B2DFF8481A898860
S31501A0135080B288426ED2DFF8800BFFB23844807922
S31501A01360DFF8181CFFB2394448717F1CEBE7B6B20F
S31501A01370701C0721B0FBF1F201FB1200002809D075
S31501A01380B6B216F108000721B0FBF1F0DFF8041A96
S31501A01390C88007E0B6B2701C0721B0FBF1F0DFF8F8
S31501A013A0F419C8800620DFF8EC1948800120DFF87F
S31501A013B0E4190881DFF8200B0068DFF8C01B08607C
S31501A013C0DFF8B80B007910F00F0050F01000DFF82D
S31501A013D0AC1B0871DFF8BC09808880B2000ADFF86F
S31501A013E09C1B097960F30301DFF8900B0171DFF80B
S31501A013F08C0B808800F0FF00DFF898198988C9B2A4
S31501A0140050EA0120DFF8741B88800820DFF86C1BE6
S31501A01410087300200700FFB2062F0BD2DFF8B80A27
S31501A01420FFB238448079DFF8541BFFB23944887182
S31501A014307F1CF0E7012000F018FE9020DFF8541978
S31501A014400870DFF8380B017BDFF8382BC9B2DFF85B
S31501A014502C0B006800F021F8F1BD38B504000D0091
S31501A014602900C9B2200000F09CFE31BD38B50400A8
S31501A014700D00290089B22000C046C04631BDF8B58D
S31501A0148004000D0016001F003B00DBB2320092B231
S31501A014902900200000F095FEF1BD2DE9FF410400D1
S31501A014A00D001600DFF84C0C046000940020070024
S31501A014B038002900C0B2C9B288420FD2FFB2F05D8E
S31501A014C08046DFF8300CFFB2384480F804806846C5
S31501A014D0FFB2384480F808807F1CE9E701208DF827
S31501A014E007002F00FFB2082F0CD2AA20DFF8041C98
S31501A014F0FFB239440871AA206946FFB2394408727D
S31501A015007F1CEFE708208DF80600684601F03AF93E
S31501A015100120DFF8E01B0873BDE8FF812DE9FF413B
S31501A0152004000D00160000940020070038002900D1
S31501A01530C0B2C9B2884209D2FFB2F05D8046684600
S31501A01540FFB2384480F808807F1CEFE702208DF8AF
S31501A0155007002F00FFB2082F06D2AA206946FFB2C4
S31501A01560394408727F1CF5E708208DF80600684605
S31501A0157001F008F9BDE8FF8138B504000D00DFF8D8
S31501A01580740B0068A04279D1EDB2012D76D1DFF8B6
S31501A015900408007820284FD0212855D022285BD0D6
S31501A015A0902802D091281AD068E0DFF8E807C08811
S31501A015B001280CD10020DFF8DC17087000F096FD99
S31501A015C00021DFF814090068FFF747FF06E00320B2
S31501A015D000F04BFDA020DFF8BC1708704EE0DFF845
S31501A015E0B4070089401CDFF8AC170881DFF8A4070F
S31501A015F00089DFF8A017C98888420CD10020DFF83E
S31501A016009417087000F072FD0021DFF8CC0800687D
S31501A01610FFF723FF0FE0DFF87C07807A002807D0C9
S31501A0162000F064FDDFF86C07007B00F065FD02E0C9
S31501A01630032000F01AFD21E0062000F016FD11207E
S31501A01640DFF85017087019E0062000F00EFD1120F2
S31501A01650DFF84017087011E00020DFF8381708708E
S31501A0166000F044FD0923DFF8E80A8288DFF8E41ACE
S31501A01670DFF8DC0A0068FFF702FFFFE731BD30B4EF
S31501A01680DFF8D44A94F88040082C44D2DFF8C84A3F
S31501A01690DFF8C45A95F881502D016051002423002A
S31501A016A01C000D00E4B2EDB2AC420ED2DFF8A84A9E
S31501A016B0DFF8A45A95F881502D012C44DBB21C44C5
S31501A016C0DBB2D55C25715B1CEAE7DFF88C4ADFF853
S31501A016D0885A95F881502D012C442173DFF8784A58
S31501A016E094F88040641CDFF8705A85F88040DFF8D2
S31501A016F0684A94F88140641CDFF85C5A85F88140F9
S31501A01700DFF8544A94F88140082C04D30024DFF86A
S31501A01710485A85F8814030BC704780B500F029F859
S31501A01720DFF8380A407B002822D0DFF8300A00799A
S31501A01730C0B20009002805D002280BD005D3032882
S31501A017400DD00FE000F06BF80EE000F0D1F800F03C
S31501A017508FFA09E000F04FF900F08AFA04E000F0F0
S31501A01760E1F901E0C046C0460020DFF8F019487350
S31501A0177001BDDFF8E41991F8801000294ED0DFF8F9
S31501A01780D819DFF8D42992F8822012018958DFF8F6
S31501A01790CC29116000210800C0B2082811D2DFF8B7
S31501A017A0B819DFF8B42992F8822012011144C0B207
S31501A017B001440979DFF8A429C0B202441171401C81
S31501A017C0EAE7DFF89419DFF8902992F8822012014E
S31501A017D01144097BDFF8842911730121DFF87C29E3
S31501A017E05173DFF8741991F88010491EDFF8682942
S31501A017F082F88010DFF8601991F88210491CDFF891
S31501A01800582982F88210DFF8501991F88210082918
S31501A0181004D30021DFF8402982F88210704738B539
S31501A01820DFF870050078000661D4DFF8300900689A
S31501A018300500DFF860050078002803D0DFF820094D
S31501A01840854254D1DFF81409007910F00F00040085
S31501A018502000DFF80819097BC0B2884247D2DFF819
S31501A01860FC08007B082842D1DFF8F008007910F0C7
S31501A018700F0000283BD0DFF8E408007910F00F0034
S31501A01880082834D2DFF8D4080068DFF8C418086045
S31501A01890DFF8C808007910F00F00DFF8B4188880C7
S31501A018A0002004002000C0B2DFF8A418898880B205
S31501A018B088420BD2DFF8A408E4B220444079DFF8CD
S31501A018C09018E4B221448871641CEBE70020DFF88C
S31501A018D0C414087000F00AFC0023DFF8740882889B
S31501A018E0DFF87018DFF868080068FFF7C8FD31BD9A
S31501A018F038B5DFF8A004007800067BD4DFF85C08D1
S31501A019000068DFF85C18884274D1DFF85008007BC4
S31501A0191008286FD1DFF84408007910F00F00050000
S31501A019202D02DFF83808808880B255EA1025ADB2BD
S31501A01930082D5FD30120DFF85C1448700620DFF87C
S31501A0194054144880DFF84C0485800120DFF8441444
S31501A0195008810020DFF83C1488720020DFF83414D7
S31501A01960C872DFF830048088401C0721B0FBF1F271
S31501A0197001FB120000280AD0DFF81804808808307D
S31501A019800721B0FBF1F0DFF80C14C88009E0DFF8FD
S31501A0199004048088401C0721B0FBF1F0DFF8F413A2
S31501A019A0C880DFF8B8070068DFF8A4170860DFF879
S31501A019B0A007858000200400E4B2062C0BD2DFF834
S31501A019C09C07E4B220448079DFF88417E4B221446D
S31501A019D08871641CF0E7042000F047FB1020DFF8B3
S31501A019E0B4130870DFF868078188DFF86407006818
S31501A019F0FFF73CFD31BD10B5DFF89803007811283B
S31501A01A0040F08F80DFF854070068DFF8541788424A
S31501A01A1040F08780DFF84407007910F00F00DFF867
S31501A01A207413097A11F00F01884211D00020DFF852
S31501A01A306413087000F05AFB0423DFF814078288A8
S31501A01A40DFF81017DFF808070068FFF718FD68E050
S31501A01A50D0480089401CCF490881CE48807A401ED3
S31501A01A60CC498872CB480089CA49C98888421FD205
S31501A01A70DFF8E806007B082853D100200400E4B271
S31501A01A80072C11D2DFF8D406E4B220444079DFF85E
S31501A01A90C016C04A528811448871BE484088401C6D
S31501A01AA0BC494880641CEAE7062000F0DEFA38E06B
S31501A01AB0B8488088B7494988401ADFF8A016097B3B
S31501A01AC088422EDADFF89406007B082829D1002067
S31501A01AD00400B0484088AF498988884211D2DFF80E
S31501A01AE07C06E4B220444079DFF86416A94A5288FC
S31501A01AF011448871641CA7484088401CA5494880A8
S31501A01B00E7E70020A349087000F0F0FA0023DFF808
S31501A01B1040068288DFF83C16DFF834060068FFF736
S31501A01B20AEFC10BD80B5DFF83C060078A0280AD02F
S31501A01B30DFF830060078912805D0DFF8280600786E
S31501A01B40A12840F09480DFF814060068DFF810168B
S31501A01B5088420CD00921DFF880030068FFF77DFCDD
S31501A01B6000F0C4FA0020DFF8FC1508707FE0DFF86A
S31501A01B70EC05007B08280BD00921D7480068FFF7A0
S31501A01B806CFC00F0B3FA0020DFF8D81508706EE0FF
S31501A01B90DFF8C805007910F00F00002803D002284D
S31501A01BA044D036D358E0DFF8BC05407800285ED192
S31501A01BB0DFF8A8054079002804D10120DFF8A41593
S31501A01BC0487005E0DFF894054079DFF8981588722A
S31501A01BD0DFF89005007891280FD0DFF8800580798D
S31501A01BE0002806D0DFF874058079DFF87815087328
S31501A01BF003E00120DFF86C1508739120DFF8641566
S31501A01C00087000F073FADFF85C05007B00F074FA47
S31501A01C102DE0DFF850054078002828D1A120DFF873
S31501A01C2044150870032000F020FA20E0DFF83405FF
S31501A01C30407800281BD1DFF82C050078A0280AD10E
S31501A01C400821A5480068FFF708FC00F04FFA00201C
S31501A01C50DFF8101508700AE005219F480068FFF714
S31501A01C60FCFB00F043FA0020DFF8F814087001BD70
S31501A01C7080B548480078102847D1DFF8D404808879
S31501A01C80FB280DD3DFF8E004007910F0F00050F046
S31501A01C900200DFF8D414087122203E4908700AE038
S31501A01CA0DFF8C404007910F0F000DFF8BC14087165
S31501A01CB0202038490870DFF8B404DFF8AC140860B6
S31501A01CC0DFF8A404007910F00F0050F03000DFF81F
S31501A01CD0981408712F48807ADFF88C144871002077
S31501A01CE0DFF8841488710320DFF87C1408730220BE
S31501A01CF000F0BBF9DFF87004017BA24AC9B2DFF894
S31501A01D0068040068FFF7C9FB42E022480078112861
S31501A01D103ED12048807A00283AD11E484078002832
S31501A01D2036D100201B498872DFF83C04007910F0F7
S31501A01D30F000DFF834140871202016490870DFF886
S31501A01D402C04DFF824140860DFF81C04007910F0D5
S31501A01D500F0050F03000DFF8101408710D48807A9A
S31501A01D60DFF8041448710020DFF8FC138871032002
S31501A01D70DFF8F4130873022000F077F9DFF8E8031F
S31501A01D80017B804AC9B2DFF8E0030068FFF785FB53
S31501A01D9001BD0000743D000038B5DFF8C803007826
S31501A01DA0912840F0968000F0C7F9012840F0918073
S31501A01DB0DFF8BC030068714908607048007910F02B
S31501A01DC00F0050F020006D490871DFF898030089D3
S31501A01DD06A49097960F3030168480171DFF8840350
S31501A01DE0807A401EDFF87C138872DFF878030089B9
S31501A01DF0DFF87013C988491E884227D208205F4997
S31501A01E00087300200400E4B2072C13D2DFF86003A4
S31501A01E10DFF850134988084480795849E4B221442F
S31501A01E204871DFF840034088401CDFF8381348802A
S31501A01E30641CE8E7012000F018F95048017B514ADB
S31501A01E40C9B24E480068FFF728FB42E0DFF8140349
S31501A01E500089DFF81013C988491E88422FD1DFF8FF
S31501A01E6004038088DFF8FC124988401A0500681C23
S31501A01E70424908730020040020002900C0B2C9B25B
S31501A01E80884210D2DFF8E802B64949880844807929
S31501A01E903A49E4B221444871B2484088401CB1494C
S31501A01EA04880641CE8E7012000F0DFF83348017B95
S31501A01EB0344AC9B231480068FFF7EFFA09E000F0E9
S31501A01EC015F90020A74908700921A9480068FFF75C
S31501A01ED0C4FA31BD00000000743C0000284A1288F3
S31501A01EE010000200264B5B8892B29A4245D0244A42
S31501A01EF0528803009BB29A4204D2214A5288821A7E
S31501A01F00110003E01E4A5288821A11001C4A508011
S31501A01F101B4A127B002A12D0194A5268002A0ED0F7
S31501A01F2089B2174A5268914206D2154A526889B2B5
S31501A01F30521A134B5A6002E00022114B5A60104A02
S31501A01F40527B022A19D10E4A9268002A0ED089B272
S31501A01F500B4A9268914206D2094A926889B2521AEC
S31501A01F60074B9A6002E00022054B9A60044A9268E8
S31501A01F70002A02D10122024B5A737047643B00002A
S31501A01F80843D0000683B000080B57A48406800287F
S31501A01F9066D17848007B012809D05FD3032823D0D6
S31501A01FA012D305283DD02CD3062847D056E06D483C
S31501A01FB00078002807D000206A49087001216C48E2
S31501A01FC00068FFF74AFA49E06648007800280AD077
S31501A01FD000206449087001235D4882885D495C48F8
S31501A01FE00068FFF74CFA39E05E480078002807D070
S31501A01FF000205C49087002215D480068FFF72DFAB0
S31501A020002CE05848007800280AD0002055490870CD
S31501A0201009234F4882884F494D480068FFF72FFA98
S31501A020201CE050480078002807D000204D490870D0
S31501A0203009214F480068FFF710FA0FE049480078D8
S31501A0204000280AD000204749087003234048828807
S31501A0205040493F480068FFF712FAFFE700F046F84B
S31501A0206001BD00203F4948737047C0B2012809D07D
S31501A0207035D3032816D00DD3052822D019D3062887
S31501A0208026D02CE001213B4A117346F2A811394A08
S31501A0209051602AE00221374A117346F2A811354A46
S31501A020A0516022E00321334A11733349314A516009
S31501A020B01BE004212F4A117342F228312D4A5160A7
S31501A020C013E005212B4A117300212A4A51600CE025
S31501A020D00621284A11732949264A516005E00021A3
S31501A020E0244A11730021234A5160704700202149D7
S31501A020F008737047443B0000C0B2802807D2C0B223
S31501A021004FF47A7101FB00F11A4A916010E0C0B256
S31501A02110F1280AD3C0B2FA2807D2C0B210F00F0133
S31501A0212064225143134A916002E01549114A916014
S31501A021300221104A517370470E49497B0800C0B26B
S31501A02140012802D100210B4A5173C0B27047000089
S31501A02150743B00007A3B0000C03A0000543B0000EB
S31501A02160F117DA18743D0000643B000017F1DA1884
S31501A02170743C0000843D0000F8240100F0490200EF
S31501A0218018F0010080B500F07EF801BD70B504001D
S31501A021900D001600320092B229002000FFF75EF86A
S31501A021A070BD38B504000D00EDB2002D04D100219B
S31501A021B0200000F029F803E00121200000F024F816
S31501A021C031BDF8B504000D0016001F00FFB2002FA7
S31501A021D007D10023320092B22900200000F021F895
S31501A021E006E00123320092B22900200000F019F87E
S31501A021F0F1BD70B504000D001600320092B229009F
S31501A022002000FFF7C3FF70BD38B504000D00DFF84D
S31501A022105003844204D1EDB2012D01D1FFF721FF74
S31501A0222031BD2DE9F04104000D0016001F00FFB2DB
S31501A02230002F21D10120DFF82C1381F80001DFF84E
S31501A0224024030460701EDFF81C13A1F8FE00002011
S31501A0225080464046310080B289B2884211D21FFA27
S31501A0226088F815F80800DFF8FC121FFA88F841442F
S31501A02270087118F10108ECE7FFB2012F01D1FFF7B0
S31501A02280F0FEBDE8F08100B583B000208DF8040012
S31501A02290B44890F80001002800F0008100F0B7FBD7
S31501A022A0B0480068B049884240F09980AD480079AD
S31501A022B0102816D011281DD0222824D027282BD0AB
S31501A022C0282832D02E2839D0312840D0342850D0D1
S31501A022D0362857D037285ED03E2841D0852863D0EE
S31501A022E06BE0A24A9F48B0F8FE109E48006800F035
S31501A022F04BFFCFE09D4A9B48B0F8FE109948006875
S31501A0230001F0B2F8C6E0994A9648B0F8FE10954891
S31501A02310006801F07FF9BDE0944A9248B0F8FE103A
S31501A023209048006801F09CFAB4E0904A8D48B0F854
S31501A02330FE108C48006801F04FFCABE08B4A89483F
S31501A02340B0F8FE108748006801F016FDA2E0874AA2
S31501A023508448B0F8FE108348006801F09FFD99E01B
S31501A02360824A8048B0F8FE107E48006802F05EF806
S31501A0237090E07E4A7B48B0F8FE107A48006802F0E9
S31501A02380DFF887E0794A7748B0F8FE10754800680B
S31501A0239002F0FCF87EE0754A7248B0F8FE1071486A
S31501A023A0006802F0F5FB75E0704A6E48B0F8FE10C1
S31501A023B06C48006802F0B2FC6CE06A4800686C499F
S31501A023C088420BD011208DF8040001A800900123AA
S31501A023D0634A01216348007900F061F85AE0614837
S31501A023E000686349884255D15E48007910280AD011
S31501A023F0112811D0222818D028281FD03E2826D04F
S31501A0240085282DD035E0594A5648B0F8FE105548D2
S31501A02410006800F0B9FE3DE0544A5248B0F8FE10FB
S31501A024205048006801F020F834E0504A4D48B0F811
S31501A02430FE104C48006801F0EDF82BE04B4A4948E4
S31501A02440B0F8FE104748006801F0C6FB22E0474AF3
S31501A024504448B0F8FE104348006801F0E7FF19E0D0
S31501A02460424A4048B0F8FE103E48006802F056FCC9
S31501A0247010E03C4800683E4988420BD011208DF8F7
S31501A02480040001A800900123354A012135480079AD
S31501A0249000F005F80020334981F8000107BD2DE9B8
S31501A024A0F84304000D0016001F00DDF82080EDB2F0
S31501A024B0002D29D02F4806607F202E4908712D486E
S31501A024C044712C48A0F8FE7000208146484629494F
S31501A024D0B1F8FE1080B288420BD21FFA89F918F81A
S31501A024E0090024491FFA89F94944887119F101099A
S31501A024F0ECE72048B0F8FE00821C92B21E491D48A6
S31501A025000068FFF776FE27E01C48066054F04000FD
S31501A025101A4908711948A0F8FE700020814648465C
S31501A025201649B1F8FE1080B288420BD21FFA89F97A
S31501A0253018F8090011491FFA89F94944487119F196
S31501A025400109ECE70D48B0F8FE00421C92B20C4915
S31501A025500A480068FFF74DFEBDE8F18300000000C0
S31501A0256017F1DA18B4430000F117DA18B9430000DD
S31501A02570F133DB18B8450000BC450000B8440000A3
S31501A02580BC44000000B5D3B09A48008845F2AA51D0
S31501A02590884200F0F5804FF48060029040F27F40BF
S31501A025A00390954800909548019040F2AB20139076
S31501A025B04FF43970149040F2AE20159040F2AF203E
S31501A025C016904FF4297017904FF42A7018904FF473
S31501A025D0367019904FF423701A9040F2B2201B90D6
S31501A025E040F2E2201C9081201D9085201E9084201F
S31501A025F01F904FF42270209040F28A20219040F241
S31501A026008920229040F2E32023904FF47E702490FB
S31501A0261040F2131025904FF40670269040F2252023
S31501A0262027904FF46070289040F2FB20299040F249
S31501A0263081202A904FF4A8702B9040F225102C905F
S31501A0264040F22F102D9040F291102E9040F2EB10F7
S31501A026502F904FF4647030904FF4D87031904FF4AE
S31501A02660387032904FF4D97033904FF48A70349009
S31501A026704FF4D170359040F2A31036904FF4D37039
S31501A02680379040F2A710389040F2F12039904FF4DC
S31501A02690F9703A904FF45C703B904FF4F8703C900F
S31501A026A040F285203D9040F286203E904FF4217065
S31501A026B03F9040F28720409040F2CD2041904FF4C8
S31501A026C03F70429040F27920439040F2FD20449021
S31501A026D04FF4327045904FF4087046904FF4147041
S31501A026E047904FF43D7048904FF45570499040F291
S31501A026F061104A904FF4B1704B904FF4D2704C9048
S31501A027004FF405704D9040F2A5104E9040F2651021
S31501A027104F9040F2F230509040F26130519000203B
S31501A027208DF8100000208DF8180000208DF82000EB
S31501A0273002208DF8280002A80B9001208DF8300008
S31501A027400220ADF8320068460D9001208DF83800C0
S31501A027503F20ADF83A0013A80F900FF24100109058
S31501A027600FF2610011900FF25900129004A8FDF723
S31501A0277062FC00202249087045F2AA501D49088032
S31501A0278053B000BD10B5040014F10803A279E17994
S31501A0279089B22068FDF76DFF10BD000070B5040079
S31501A027A00D0016001548844202D01348844205D173
S31501A027B032002900C9B22000FEF761FF70BD0000FA
S31501A027C07047000038B504000D00EDB2002D08D108
S31501A027D0C4F3400000280CD001210A48FEF7CCFE24
S31501A027E007E0C4F34000002803D000210548FEF706
S31501A027F0C3FE31BD9A540000F117DA18F133DB1884
S31501A028001D101CB717F1DA182DE9FE4F012000F0B3
S31501A028104EF80020DFF8A818087000F09BF84FF4D6
S31501A028208870029000200190DFF89848019A0299D9
S31501A02830200002F01AEB4FF48C7000900024DFF810
S31501A02840885822000099280002F00EEBC825002620
S31501A02850DFF8787832002900380002F006EB5FF045
S31501A02860FF30DFF86018C8605FF0FF30DFF8581856
S31501A0287048605FF0FF30DFF8501888600E275FF0E0
S31501A028800008DFF84C9842463900484602F0ECEAC7
S31501A0289000F04BFB4FF49E795FF0000ADFF834B8E5
S31501A028A052464946584602F0E0EABDE8F78FC0B263
S31501A028B0012805D0C0B2022802D0C0B2032803D194
S31501A028C0DFF81418087003E00121DFF80C28117055
S31501A028D07047DFF804080078704730B4DFF8FC478A
S31501A028E02060DFF8F847A180002423001C00E4B291
S31501A028F00D00A4B2ADB2AC4208D2DBB2D45CDFF813
S31501A02900DC57DBB21D442C725B1CEFE730BC704771
S31501A029100021DFF8C82711600021DFF8C0279180C8
S31501A0292000210800C0B2FA2807D20021DFF8AC279F
S31501A02930C0B202441172401CF4E77047DFF8A00749
S31501A0294000787047DFF89C0700887047DFF880079A
S31501A02950007970470020DFF8781708700020DFF8AB
S31501A02960701748720020DFF8681788720020DFF818
S31501A029706017C8720020DFF8581708730020DFF827
S31501A02980501708710020DFF8481748710020DFF8BA
S31501A02990401788710020DFF83817C8710020DFF8CA
S31501A029A0301708727047000072B6DFF83C07DFF8EF
S31501A029B03C170860A520DFF838170870704780B566
S31501A029C0FFF787FF012821D0DFF828070078012823
S31501A029D007D10020DFF81C1708700020DFF81817B0
S31501A029E00880DFF814070088411CDFF80C27118046
S31501A029F080B2B0F5FA7F09D90020DFF8FC1608806D
S31501A02A000020DFF8F016087000F006F801BD0120DD
S31501A02A10DFF8E016087070472DE9F84F0120FFF79F
S31501A02A2046FF00F0E8F80020DFF8941608704FF48E
S31501A02A30887000900024DFF88C56220000992800A7
S31501A02A4002F012EA4FF48C750026DFF87C7632008C
S31501A02A502900380002F008EAC8275FF00008DFF86D
S31501A02A606C9642463900484602F0FEE94FF49E793B
S31501A02A705FF0000ADFF85CB652464946584602F0B6
S31501A02A80F4E95FF0FF30DFF83C16C8605FF0FF3075
S31501A02A90DFF8341648605FF0FF30DFF82C16886047
S31501A02AA00020DFF82C1608700020DFF82416087124
S31501A02AB000F004F8FFF72CFFBDE8F18F80B500F018
S31501A02AC07EF8002801D1FFF76FFF01BDE0B500F048
S31501A02AD076F8DFF828160860DFF820060068DFF828
S31501A02AE02016884206D0DFF814060068DFF814160F
S31501A02AF0884236D172B602F0F1F9FFF743FD02F032
S31501A02B005FFD62B602208DF8040000208DF8050055
S31501A02B1032208DF8060000208DF80700C8208DF818
S31501A02B2008000220DFF8B0150870002000F054F864
S31501A02B300020DFF8C81588710020DFF8C01588804D
S31501A02B40DFF8B8050068DFF8BC15884232D101A8C4
S31501A02B5000900523DFF8B02500211020FFF79FFC88
S31501A02B6028E0DFF898050068DFF8A015884210D1A3
S31501A02B700020DFF8881588710020DFF8801588808D
S31501A02B8072B602F0ABF9FFF7FDFC02F019FD62B6D1
S31501A02B9010E003F03FF9002802D000F035F801E07B
S31501A02BA000F032F872B602F099F9FFF7EBFC02F0E9
S31501A02BB007FD62B600F042F803F0FEF907BD80B545
S31501A02BC00FF261130422DFF84815012000F048F83E
S31501A02BD0DFF83C05406802BD10B50400DFF83005FA
S31501A02BE0446003F0CDFB01230422DFF82415012064
S31501A02BF000F06DF810BD0020DFF8001588710020E7
S31501A02C00DFF8F8148880704710B502F00FFD72B690
S31501A02C10BFF34F8FBFF36F8F40F6B830040020008B
S31501A02C20441E002805D0DFF8EC04DFF8EC14086098
S31501A02C30F5E7DFF8E4040068804710BD80B50FF220
S31501A02C4009130322DFF8D414022000F009F80FF2C9
S31501A02C5031131822DFF8C814032000F001F801BDD2
S31501A02C602DE9F04104000D0016001F002000C0B29E
S31501A02C7003F0D1FE80465FFA88F8B8F1010F01D1C1
S31501A02C80B84720E05FFA88F8B8F1020F1AD13200EE
S31501A02C9092B229002000C0B203F0CCFE80465FFAB2
S31501A02CA088F8B8F1000F0ED103F0AEFB012802D1CE
S31501A02CB004F06AF9F8E72868DFF86814884202D0B8
S31501A02CC0B84700E0B8474046C0B2BDE8F0812DE95B
S31501A02CD0F04104000D0016001F005FF0010820005E
S31501A02CE0C0B203F098FE002818D003F08DFB01288E
S31501A02CF002D104F049F9F8E7320092B22900200086
S31501A02D00C0B203F0D5FE8046FFB2012F06D103F073
S31501A02D107BFB012802D104F037F9F8E74046C0B29F
S31501A02D20BDE8F081DFF8FC03DFF8E41308600020BA
S31501A02D30DFF8DC1348600020DFF8D4138860002098
S31501A02D40DFF8CC13C8607047DFF8D803DFF8CC13DF
S31501A02D5008600020DFF8C413C8710020DFF8BC1397
S31501A02D6088710020DFF8B41348710020DFF8AC1396
S31501A02D70087140F2D270DFF8A41388607047000092
S31501A02D80DFF8A013DFF8982311600021DFF8902364
S31501A02D9011710021DFF88823517100210800C0B20A
S31501A02DA0102807D22021DFF87823C0B202449171FE
S31501A02DB0401CF4E73021DFF8682391713021DFF858
S31501A02DC06023D1713121DFF8582311720021080047
S31501A02DD0C0B20A2807D22021DFF84423C0B2024498
S31501A02DE09175401CF4E73821DFF834239175382119
S31501A02DF0DFF82C23D1753921DFF82423117631216F
S31501A02E00DFF81C2351763121DFF814239176322184
S31501A02E10DFF80C23D1763821DFF804231177392185
S31501A02E20DFF8FC2251773721DFF8F42291773021A0
S31501A02E30DFF8EC22D17700210800C0B2102808D211
S31501A02E402021DFF8DC22C0B2024482F82B10401CFC
S31501A02E50F3E73021DFF8C82282F82B103021B04ADF
S31501A02E6082F82C103021AE4A82F82D103721AC4AB7
S31501A02E7082F82E103221AA4A82F82F103121A84AAF
S31501A02E8082F830103121A64A82F831104321A44A92
S31501A02E9082F832103221A24A82F833103021A04A98
S31501A02EA082F834102F219E4A82F8351041219C4A7E
S31501A02EB082F8361041219A4A82F83710002108007B
S31501A02EC0C0B2102807D22021954AC0B2024482F886
S31501A02ED03B10401CF4E73021914A82F83B10302187
S31501A02EE08F4A82F83C1033218D4A82F83D10002189
S31501A02EF00800C0B2102807D22021894AC0B20244D4
S31501A02F0082F84B10401CF4E72021854A82F85B1019
S31501A02F100021834A82F85C100121814A82F85D1062
S31501A02F2001217F4A82F85E10704700207E49887091
S31501A02F3000207D490880704738B504002500280087
S31501A02F40451E80B2002802D004F01EF8F7E731BD75
S31501A02F5030B45FF0FF335B4CE36002000B00591EF7
S31501A02F60002B10D0714B574CE46815786C4004F0D7
S31501A02F70FF0453F82430534CE46893EA1423514CCC
S31501A02F80E360521CEAE730BC704730B402000B0084
S31501A02F90591E002B10D0654B4B4C646815786C40BC
S31501A02FA004F0FF0453F82430474C646893EA1423D1
S31501A02FB0454C6360521CEAE730BC704710B401006F
S31501A02FC05A4A414B9B680C78634003F0FF0352F8C1
S31501A02FD023203D4B9B6892EA13223B4B9A6010BC7F
S31501A02FE0704738B500200400E4B20A2C67DA3748E6
S31501A02FF0E4B2142101FB04F1405C01285DD1334800
S31501A03000E4B2142101FB04F108444068B0F1D17F78
S31501A030100ED12E48E4B2142101FB04F10844406804
S31501A0302010302A49E4B2142202FB04F2114448608A
S31501A030302648E4B2142101FB04F10844406823495F
S31501A03040E4B2142202FB04F21144C968884234D2C4
S31501A030501E48E4B2142101FB04F10844406803F0C0
S31501A0306067F8050028008DF803000DF10300FFF7AE
S31501A03070A5FF280A8DF802000DF10200FFF79EFFB9
S31501A03080280C8DF801000DF10100FFF797FF280E1E
S31501A030908DF800006846FFF791FF0C48E4B21421B1
S31501A030A001FB04F108444068001D0849E4B214225A
S31501A030B002FB04F211444860BAE7641C94E731BDEF
S31501A030C0A6540000743F000084400000EC420000BA
S31501A030D0F03E0000B0410000AC3A0000EC3D00001B
S31501A030E0A4540000A054000055CEAC5C000060B012
S31501A030F0820360B0A5540000AA3A00006C3F00000C
S31501A03100633658853663855817F1DA18A35A7AA714
S31501A03110A04100001000A201E83D0000003F000010
S31501A031200C3F00005AA5A77A9C410000409AA00135
S31501A031302DE9F0415FF0D17002F0FAFF0400200002
S31501A031400500200A0600200C0700200E80464346F3
S31501A03150DBB23A00D2B23100C9B22800C0B200F047
S31501A0316004F804002000BDE8F08130B40400E4B204
S31501A03170C9B20D0455EA0465D2B255EA0225DBB2FD
S31501A031801D43280030BC7047F8B504000D00160099
S31501A031900027002007003200290089B22000FFF78E
S31501A031A09CFBFFB2002F02D10020C0B20700FFB2E4
S31501A031B0002F02D10020C0B20700FFB2002F02D11A
S31501A031C003F040FF0700FFB2002F02D10020C0B2DA
S31501A031D00700FFB2002F02D103F04FFF0700FFB295
S31501A031E0002F02D10020C0B20700FFB2002F01D1EB
S31501A031F000F003F8FFF78CFBF1BD10B50024E4B293
S31501A03200002C02D103F054FF0400E4B2002C02D139
S31501A0321003F0A1FF0400E4B2002C02D103F0C9FF20
S31501A032200400E4B2002C02D10020C0B20400E4B232
S31501A03230002C02D104F00AF80400E4B2002C02D159
S31501A032400020C0B20400E4B2002C02D10020C0B21A
S31501A032500400E4B2002C13D17A48007A10F07F0062
S31501A03260012804D00CD3032807D003D308E000F02B
S31501A0327008F805E000F096F802E000F0BBF8FFE7D9
S31501A0328010BD2DE9F04F85B00120FFF710FBFFF728
S31501A03290B2FC00206C4908704FF48870039000249A
S31501A032A06A4D22000399280001F0DEED4FF48C75DA
S31501A032B00026674F32002900380001F0D6EDC82755
S31501A032C05FF00008DFF88C9142463900484601F0CC
S31501A032D0CCED5FF0FF305D49C8605FF0FF305C491F
S31501A032E048605FF0FF305A49886000205A4908704B
S31501A032F00020594908714FF49E795FF0000ADFF862
S31501A033005CB152464946584601F0AEED4D48007AA9
S31501A03310C0B2C009C0B2002839D1002049494872BB
S31501A0332032204849887200204649C872C8204549BA
S31501A03330087306208DF8040050208DF805000120A1
S31501A033408DF806003F48407A8DF807003D48807AFF
S31501A033508DF808003B48C07A8DF809003948007BF2
S31501A033608DF80A00AA208DF80B0001AA08213C4875
S31501A03370FEF7D4F8FFF723FC0090009800280ED1A1
S31501A0338042F21070FFF7D8FDFFF70EFB07E0FFF73B
S31501A0339016FC00900098002801D1FFF705FB05B0A7
S31501A033A0BDE8F08F80B50220FFF781FA00202A49F7
S31501A033B00870002028490871FFF71DFC2148007AF2
S31501A033C0C0B2C009C0B2002813D100201D4948725D
S31501A033D032201C49887200201A49C872C82019498E
S31501A033E008732048009005231D4A00211020FFF7ED
S31501A033F056F801BD80B50320FFF759FA00201649FA
S31501A034000870002014490871FFF7F5FB0D48007AF2
S31501A03410C0B2C009C0B2002813D100200949487220
S31501A0342032200849887200200649C872C820054979
S31501A0343008730C4800900523094A00211020FFF7C4
S31501A034402EF801BDEC3D0000A6540000743F00001B
S31501A0345084400000EC420000F03E0000B0410000B4
S31501A0346017F1DA18F43D0000F8B504000D001600B6
S31501A0347000273200290089B22000FFF72EFAFFB2F9
S31501A03480002F02D103F03EFF0700FFB2002F02D1A9
S31501A034900020C0B20700FFB2002F02D103F052FFF5
S31501A034A00700FFB2002F02D10020C0B20700FFB271
S31501A034B0002F02D103F061FF0700FFB2002F02D156
S31501A034C00020C0B20700FFB2002F01D100F003F81F
S31501A034D0FFF71EFAF1BD10B50024E4B2002C02D10B
S31501A034E003F066FF0400E4B2002C02D103F09AFFB8
S31501A034F00400E4B2002C02D10020C0B20400E4B260
S31501A03500002C02D10020C0B20400E4B2002C02D1EA
S31501A0351003F0B0FF0400E4B2002C02D10020C0B237
S31501A035200400E4B2002C02D10020C0B20400E4B22F
S31501A03530002C0FD13548007A10F07F00C0B20128C7
S31501A0354002D0032803D005E000F005F802E000F060
S31501A035502FF8FFE710BD00B583B02C48007AC0B2A2
S31501A03560C009C0B2002820D102208DF80000512048
S31501A035708DF8010001208DF80200AA208DF8030024
S31501A03580AA208DF80400AA208DF80500AA208DF89E
S31501A035900600AA208DF807006A4608211C48FDF7F7
S31501A035A07CFF42F21070FFF7C7FCFFF7FDF907BDDC
S31501A035B000B583B01548007AC0B2C009C0B20028D0
S31501A035C020D102208DF8000051208DF801000320A2
S31501A035D08DF80200AA208DF80300AA208DF8040018
S31501A035E0AA208DF80500AA208DF80600AA208DF83C
S31501A035F007006A4608210648FDF74FFF42F2107000
S31501A03600FFF79AFCFFF7D0F907BD0000EC3D0000DB
S31501A0361017F1DA18F8B504000D00160000273200DC
S31501A03620290089B22000FFF758F9FFB2002F02D175
S31501A036300020C0B20700FFB2002F02D10020C0B205
S31501A036400700FFB2002F02D103F056FF0700FFB219
S31501A03650002F02D103F06BFF0700FFB2002F02D1AA
S31501A0366003F095FF0700FFB2002F02D10020C0B2E0
S31501A036700700FFB2002F01D100F003F8FFF748F9C8
S31501A03680F1BD80B56B48007A000280B26949497ADA
S31501A03690084380B24FF40071401A12D0401E13D0D5
S31501A036A04EF67F71401A12D0801F13D0401E14D03F
S31501A036B0801E15D00A3816D0401F17D0401E18D02C
S31501A036C01AE000F053F817E000F05EF814E000F0FD
S31501A036D069F811E000F079F80EE000F084F80BE04B
S31501A036E000F094F808E000F008F805E000F018F8FA
S31501A036F002E000F028F8FFE701BD70B582B0102402
S31501A037004D4D4E4E22002900300003F07EEF4C486D
S31501A03710009012234B4A00212220FEF7C0FE73BD62
S31501A0372070B582B01024484D444E220029003000C5
S31501A0373003F06AEF424800901223424A0021222058
S31501A03740FEF7ADFE73BD70B582B004243F4D3B4E6E
S31501A0375022002900300003F058EF394800900623D3
S31501A03760384A00212220FEF79AFE73BD80B538485B
S31501A03770007930498872324800900323314A0021EA
S31501A037802220FEF78CFE01BD80B53148407929493A
S31501A0379088722B48009003232A4A00212220FEF793
S31501A037A07EFE01BD70B582B010242A4D234E2200A3
S31501A037B02900300003F028EF214800901223214A66
S31501A037C000212220FEF76BFE73BD80B5FFF781F8BD
S31501A037D0184988721A48009003231A4A0021222008
S31501A037E0FEF75DFE01BD70B582B015241A4D134ECC
S31501A037F022002900300003F008EF1148009017239A
S31501A03800104A00212220FEF74AFE73BD70B582B090
S31501A038101024124D094E22002900300003F0F4EEC7
S31501A03820074800900C23074A00212220FEF737FE05
S31501A0383073BD0000EC3D0000473F0000F63D0000CF
S31501A03840F43D000017F1DA18573F0000673F00006A
S31501A038500C3F0000123F0000223F0000373F00004E
S31501A03860F8B504000D00160000273200290089B220
S31501A038702000FFF732F8FFB2002F02D103F02EFF8E
S31501A038800700FFB2002F02D10020C0B20700FFB28D
S31501A03890002F02D103F044FF0700FFB2002F02D18F
S31501A038A00020C0B20700FFB2002F02D10020C0B293
S31501A038B00700FFB2002F02D10020C0B20700FFB25D
S31501A038C0002F01D100F003F8FFF722F8F1BD10B5E2
S31501A038D00024E4B2002C02D103F03DFF0400E4B2BF
S31501A038E0002C02D103F071FF0400E4B2002C02D136
S31501A038F003F093FF0400E4B2002C02D10020C0B271
S31501A039000400E4B2002C02D103F0D7FF0400E4B214
S31501A03910002C02D104F00BF80400E4B2002C02D171
S31501A039200020C0B20400E4B2002C02D104F024F8B5
S31501A039300400E4B2002C0FD19F48007A10F07F005A
S31501A03940C0B2112802D0122803D005E000F005F874
S31501A0395002E000F096F8FFE710BD1CB500200400B8
S31501A039609648007901283CD094480078012821D0B6
S31501A0397002F018FB9248006890F0310010308F4990
S31501A0398048718F480068000A90F0560009308B49AB
S31501A0399088718B480068000C90F08700401C87490D
S31501A039A0C87187480068000E90F0920015308349CF
S31501A039B0087204E083488079401C8249887102F02C
S31501A039C0DFFC012303227F490220FFF780F97D480E
S31501A039D08079032801D302F034FB012077490870CE
S31501A039E00BE00020754948710020744988710020B8
S31501A039F07249C871002071490872704840796E49B0
S31501A03A0048726E4880796C4988726C48C0796A4957
S31501A03A10C8726A48007A68490873684840798DF87F
S31501A03A200400664880798DF805006448C0798DF850
S31501A03A3006006248007A8DF807009DF80400002868
S31501A03A400BD19DF80500002807D19DF80600002896
S31501A03A5003D19DF80700002803D05B4901A800F017
S31501A03A6071F85548007AC0B2C009C0B2002807D182
S31501A03A70564800900523564A00212720FEF70FFD40
S31501A03A8013BD38B54C48407A05004B48807A50EAB8
S31501A03A9005254948C07A50EA05254748007B50EAE2
S31501A03AA005254648407A04004448807A50EA042411
S31501A03AB04248C07A50EA04244048007B50EA0424D4
S31501A03AC0A54223D101203D49087100203B49087038
S31501A03AD000203C49487100203A49887102F050FC07
S31501A03AE00123032237490220FFF7F1F83248007A71
S31501A03AF0C0B2C009C0B2002823D134480090012326
S31501A03B00334A00212720FEF7CAFC1AE02D48807906
S31501A03B10401C2C49887102F033FC01230322294958
S31501A03B200220FFF7D4F827488079032804D302F0AE
S31501A03B3088FA03F03CFF04E000202049087003F056
S31501A03B4049FF31BD18B400231A0092B2042A0AD241
S31501A03B5092B2835C1F4C92B2A45C63406C4692B253
S31501A03B60A354521CF1E79DF802309DF80340E4B23C
S31501A03B70A40854EA83130B709DF803309DF8004006
S31501A03B8014F03F0454EA83134B709DF8003013F0F0
S31501A03B90FC039DF80140E4B253EA94138B709DF89F
S31501A03BA0013013F0FC039DF8024014F003042343F3
S31501A03BB0CB7011BC70470000EC3D0000F03E000048
S31501A03BC0A03A0000003F0000F93E0000F43D0000CD
S31501A03BD017F1DA187CA7A001F8B504000D001600AC
S31501A03BE000273200290089B22000FEF776FEFFB237
S31501A03BF0002F02D10020C0B20700FFB2002F02D1D0
S31501A03C0003F004FF0700FFB2002F02D10020C0B2CB
S31501A03C100700FFB2002F02D103F01BFF0700FFB27E
S31501A03C20002F02D103F032FF0700FFB2002F02D10D
S31501A03C3003F057FF0700FFB2002F02D103F06CFF7C
S31501A03C400700FFB2002F01D100F003F8FEF760FED6
S31501A03C50F1BD10B50024E4B2002C02D103F088FF17
S31501A03C600400E4B2002C02D103F0EEFF0400E4B29A
S31501A03C70002C02D10020C0B20400E4B2002C02D173
S31501A03C8004F016F80400E4B2002C02D104F038F8CE
S31501A03C900400E4B2002C02D10020C0B20400E4B2B8
S31501A03CA0002C02D10020C0B20400E4B2002C17D12E
S31501A03CB02E48007A10F07F00002805D0022809D0EE
S31501A03CC005D3032809D00BE000F00BF808E000F0BB
S31501A03CD019F805E000F027F802E000F035F8FFE753
S31501A03CE010BD80B52148007AC0B2C009C0B2002873
S31501A03CF007D11F48009001231E4A00212820FEF764
S31501A03D00CEFB01BD80B51948007AC0B2C009C0B2C8
S31501A03D10002807D1164800900123164A0021282021
S31501A03D20FEF7BDFB01BD80B51048007AC0B2C0093F
S31501A03D30C0B2002807D10E48009001230D4A0021E8
S31501A03D402820FEF7ACFB01BD80B50848007AC0B2B9
S31501A03D50C009C0B2002807D1054800900123054A31
S31501A03D6000212820FEF79BFB01BD0000EC3D0000D1
S31501A03D70F43D000017F1DA18F8B504000D0016009D
S31501A03D8000273200290089B22000FEF7A6FDFFB266
S31501A03D90002F02D104F028F80700FFB2002F02D1AC
S31501A03DA004F042F80700FFB2002F02D104F057F841
S31501A03DB00700FFB2002F02D104F06CF80700FFB292
S31501A03DC0002F02D104F096F80700FFB2002F02D10E
S31501A03DD00020C0B20700FFB2002F01D100F003F806
S31501A03DE0FEF796FDF1BD80B52548007A000280B2A6
S31501A03DF02349497A084380B24FF29811401A02D05A
S31501A03E00401E03D005E000F005F802E000F01DF821
S31501A03E10FFE701BD70B582B010241A4D1A4E2200DB
S31501A03E202900300003F0F0EB02F0AAFA01231822D0
S31501A03E3016490320FEF74BFF154800900223154AA9
S31501A03E4000212E20FEF72BFB73BD70B582B0042492
S31501A03E500C4D114E22002900300003F0D6EB02F0E2
S31501A03E608FFA0123182209490320FEF730FF0848DB
S31501A03E7000900223074A00212E20FEF710FB73BDF6
S31501A03E80EC3D0000F63D0000573F00000C3F00004E
S31501A03E90F43D000017F1DA18673F0000F8B50400F9
S31501A03EA00D00160000273200290089B22000FEF776
S31501A03EB014FDFFB2002F02D104F05AF80700FFB299
S31501A03EC0002F02D104F074F80700FFB2002F02D12F
S31501A03ED004F089F80700FFB2002F02D104F09EF882
S31501A03EE00700FFB2002F02D104F0C8F80700FFB205
S31501A03EF0002F02D104F020F90700FFB2002F01D153
S31501A03F0000F003F8FEF704FDF1BD2DE9FF41002005
S31501A03F108DF8040000208DF80400DFF8E804407A4B
S31501A03F20000280B2DFF8DC14897A084380B240F23D
S31501A03F300221401A08D04FF6FE41401A00F0D28065
S31501A03F40401E00F092815BE2DFF8BC0440780128B4
S31501A03F5058D1DFF8B004C07ADFF8A814097B0904A8
S31501A03F6051EA0060DFF89C14497B50EA0120DFF892
S31501A03F709414897B084307005FF0FF304740DFF8C0
S31501A03F808C044068B8421ED10120DFF8781408726B
S31501A03F900220DFF8701448720220DFF868148872D4
S31501A03FA00420DFF86014C8720120DFF8601448709D
S31501A03FB0DFF85C0400900423DFF8582400213120A7
S31501A03FC0FEF76DFA8DE00120DFF8381408720220A1
S31501A03FD0DFF8301448720220DFF828148872052011
S31501A03FE0DFF82014C8720020DFF820144870DFF82B
S31501A03FF0200400900423DFF81C2400213120FEF7C1
S31501A040004EFA6EE09DF8040000286AD1DFF8F803A5
S31501A04010B0F80C0100280BD122208DF8040001A8CC
S31501A0402000900123DFF8EC2301213120FEF737FAB6
S31501A040309DF80400002854D1DFF8C803C07ADFF840
S31501A04040C413097B090451EA0060DFF8B813497B60
S31501A0405050EA0120DFF8AC13897B08430700DFF89B
S31501A04060A8038168DFF8B003FEF772FF5FF0FF30A7
S31501A040704740DFF89403C068B8421ED10120DFF89B
S31501A04080841308720220DFF87C1348720220DFF83D
S31501A04090741388720420DFF86C13C8720120DFF84C
S31501A040A068134870DFF8680300900423DFF86423DF
S31501A040B000213120FEF7F3F913E00120D14908725E
S31501A040C00220D04948720220CE4988720520CD49E6
S31501A040D0C872CF4800900423CE4A00213120FEF7B2
S31501A040E0DEF98DE19DF8040000280ED1C64840787E
S31501A040F001280AD022208DF8040001A800900123EE
S31501A04100C44A01213120FEF7CAF99DF8040000280E
S31501A0411033D1BC48007BBB49497B090451EA006005
S31501A04120B849897B50EA0120B649C97B08430400F6
S31501A04130B448007CB349497C090451EA0060B149FD
S31501A04140897C50EA0120AF49C97C08430500B4F136
S31501A04150D17F02D1B5F5E81F0FD331208DF8040028
S31501A04160A8480068AD49884207D101A8009001235B
S31501A04170A84A01213120FEF792F99DF804000028F2
S31501A0418072D103208DF808007F208DF80900312017
S31501A041908DF80A0078208DF80B00AA208DF80C0066
S31501A041A0AA208DF80D00AA208DF80E00AA208DF860
S31501A041B00F0002AA08219748FDF7B0F99848FEF723
S31501A041C00BFD02F049F85FF0D17001F04DFF002818
S31501A041D006D101209349087004208A49C87205E0D6
S31501A041E000209049087005208649C8725FF0FF300B
S31501A041F0864948608C484079FF2804D08A4840798E
S31501A04200401C8949487102F0BBF80123182286494E
S31501A042100320FEF75CFD00208046B8F57A6F05D233
S31501A0422018F1010800BF02F0AFFEF6E705208DF8F0
S31501A04230080071208DF8090001208DF80A00FF20E1
S31501A042408DF80B0000208DF80C006E48C07A8DF811
S31501A042500D00AA208DF80E00AA208DF80F0002AA43
S31501A0426008216C48FDF75AF9CAE09DF80400002818
S31501A0427023D16648407801281FD005208DF8040077
S31501A0428005208DF8080071208DF8090001208DF810
S31501A042900A00FF208DF80B0001208DF80C000520E7
S31501A042A08DF80D00AA208DF80E00AA208DF80F001A
S31501A042B002AA08215748FDF731F99DF80400002804
S31501A042C040F09D8003208DF808007F208DF809001D
S31501A042D031208DF80A0078208DF80B00AA208DF8E0
S31501A042E00C00AA208DF80D00AA208DF80E00AA2098
S31501A042F08DF80F0002AA08214648FDF70FF95FF0D5
S31501A04300FF3042498860FEF76CFE404880685FF046
S31501A04310FF3148403D498860FEF70AFF06003B4849
S31501A043208068B0423FD102F02BF80020FEF754FC82
S31501A043303D480079FF2804D03B480079401C3A4902
S31501A0434008710020384948710123182236490320F3
S31501A04350FEF7BDFC00208046B8F57A6F05D218F1AC
S31501A04360010800BF02F010FEF6E705208DF808004F
S31501A0437071208DF8090001208DF80A00FF208DF823
S31501A043800B0001208DF80C0004208DF80D00AA2049
S31501A043908DF80E00AA208DF80F0002AA08211D484B
S31501A043A0FDF7BCF82BE09DF80400002827D10020DA
S31501A043B08046B8F57A6F05D218F1010800BF02F060
S31501A043C0E3FDF6E705208DF8080071208DF80900B8
S31501A043D001208DF80A00FF208DF80B0001208DF831
S31501A043E00C0005208DF80D00AA208DF80E00AA203C
S31501A043F08DF80F0002AA08210648FDF78FF8FFE7FE
S31501A04400BDE8FF81EC3D0000743F00008440000040
S31501A04410F43D000017F1DA18853F0000F117DA180C
S31501A04420A35A7AA7A65400000C3F0000F8B50400D1
S31501A044300D00160000273200290089B22000FEF7E0
S31501A044404CFAFFB2002F02D10020C0B20700FFB282
S31501A04450002F02D10020C0B20700FFB2002F02D167
S31501A0446003F090FE0700FFB2002F02D10020C0B2D8
S31501A044700700FFB2002F02D103F09FFE0700FFB293
S31501A04480002F02D10020C0B20700FFB2002F01D138
S31501A0449000F003F8FEF73CFAF1BD10B50024E4B232
S31501A044A0002C02D103F0A4FE0400E4B2002C02D138
S31501A044B003F0BFFE0400E4B2002C02D10020C0B27A
S31501A044C00400E4B2002C02D10020C0B20400E4B280
S31501A044D0002C02D103F0CFFE0400E4B2002C02D1DD
S31501A044E00020C0B20400E4B2002C02D10020C0B268
S31501A044F00400E4B2002C08D10E48007A10F07F0027
S31501A04500002802D100F002F8FFE710BD80B5FEF742
S31501A045107EFA0848007AC0B2C009C0B2002807D105
S31501A04520054800900123054A00213E20FDF7B7FF6B
S31501A0453001BD0000EC3D0000F43D000017F1DA18C2
S31501A04540F8B504000D00160000273200290089B233
S31501A045502000FEF7C2F9FFB2002F02D103F0B2FE8E
S31501A045600700FFB2002F02D103F0D2FE0700FFB26F
S31501A04570002F02D103F0E8FE0700FFB2002F02D1FF
S31501A0458003F0FFFE0700FEF7C3F9F1BDF8B504007D
S31501A045900D00160000273200290089B22000FEF77F
S31501A045A09CF9FFB2002F02D104F002F90700FFB275
S31501A045B0002F02D10020C0B20700FFB2002F02D106
S31501A045C004F019F90700FFB2002F02D104F02FF968
S31501A045D00700FFB2002F02D10020C0B20700FFB230
S31501A045E0002F02D10020C0B20700FFB2002F01D1D7
S31501A045F000F003F8FEF78CF9F1BD2DE9FC4100208E
S31501A046008DF8040000208DF80400DFF858054078E5
S31501A04610012840F098819DF80400002815D1DFF803
S31501A0462048050078012810D0DFF83C05007802285B
S31501A046300BD024208DF8040001A800900123DFF8F7
S31501A046402C2501213620FDF72AFF9DF8040000281C
S31501A0465013D1DFF81C058088401E0400A4B2E12C0A
S31501A046600BD313208DF8040001A800900123DFF8D5
S31501A04670FC2401213620FDF712FF9DF80400002835
S31501A0468010D1DFF8F004007801280BD070208DF846
S31501A04690040001A800900123DFF8D02401213620CF
S31501A046A0FDF7FDFE9DF80400002815D1DFF8B8043A
S31501A046B0D0F80C01DFF8B014D1F8101188420BD252
S31501A046C071208DF8040001A800900123DFF89C2435
S31501A046D001213620FDF7E3FE9DF80400002840F0F5
S31501A046E0B281DFF88404007B012840F0B080DFF8B6
S31501A046F07804D0F81001002840F0A980DFF86804FA
S31501A04700007BDFF86C14097A88422FD1A4B2DFF8B6
S31501A047106874DFF8688422003900404602F074EF1D
S31501A04720DFF84404A0F80841DFF83C04D0F81001F2
S31501A04730DFF83414B1F808114018DFF82C14C1F8C9
S31501A0474010010220DFF820140870DFF81C04007B9A
S31501A04750DFF81C140872DFF8280400900123DFF8A3
S31501A047600C2400213620FDF79AFE6CE1DFF8F80350
S31501A04770007B401CDFF8F813097A88425AD1DFF88A
S31501A04780E8030078022855D1DFF8DC03B0F8081158
S31501A04790DFF8E80300F059F90500EDB2002D3CD190
S31501A047A0DFF8C403D0F81001DFF8BC13B1F8081183
S31501A047B04018DFF8B413C1F81001A4B2DFF8B8733A
S31501A047C0DFF8B88322003900404602F01EEFDFF879
S31501A047D09803A0F80841DFF89003D0F8100110FA69
S31501A047E084F0DFF88413C1F81001DFF87C03007BA5
S31501A047F0401CDFF874130873DFF86C03007BDFF845
S31501A0480070130872DFF8780300900123DFF85C23A8
S31501A0481000213620FDF743FE15E172208DF8040034
S31501A0482001A800900123DFF8442301213620FDF7DA
S31501A0483036FE08E173208DF8040001A8009001233B
S31501A04840DFF8282301213620FDF729FEFBE0C64823
S31501A04850007BC749097A88421FD1C348007802283C
S31501A048601BD1A4B2C44FDFF81483220039004046FD
S31501A0487002F0CAEEBC48A0F808410220BA49087065
S31501A04880B948007BBA494872BD4800900123B74A8E
S31501A0489000213620FDF703FED5E0B348007B401C7E
S31501A048A0B349097AC0B2884241D1AF4800780228FB
S31501A048B03DD1AD48B0F80811B04800F0C6F80500E2
S31501A048C0EDB2002D27D1A4B2AB4FDFF8B082220002
S31501A048D03900404602F098EEA348A0F80841A24844
S31501A048E0D0F81001A049B1F8081140189E49C1F8A5
S31501A048F010019D48007B401C9B4908739A48007B88
S31501A049009B4948729E4800900123984A002136206F
S31501A04910FDF7C5FD97E072208DF8040001A800906F
S31501A049200123924A01213620FDF7B9FD8BE07320C0
S31501A049308DF8040001A8009001238C4A012136209C
S31501A04940FDF7ADFD7FE09DF80400002812D1854852
S31501A04950007801280ED08348007802280AD02420A6
S31501A049608DF8040001A800900123804A0121362078
S31501A04970FDF795FD9DF80400002864D17948007CD7
S31501A049807B49097A88423BD179488088401E040038
S31501A04990A4B2202C0AD013208DF8040001A80090FF
S31501A049A00123724A01213620FDF779FD9DF8040005
S31501A049B0002848D120206B49A1F80C01002006004F
S31501A049C03000210080B289B2884209D26848B6B2C5
S31501A049D03044407A6349B6B231444874761CEFE755
S31501A049E00220604908705F48007C614908726448EA
S31501A049F0009001235D4A00213620FDF750FD22E0FB
S31501A04A009DF8040000280FD15648B0F80C012028C3
S31501A04A100AD113208DF8040001A800900123534A5E
S31501A04A2001213620FDF73BFD9DF8040000280AD19F
S31501A04A3073208DF8040001A8009001234B4A01219F
S31501A04A403620FDF72CFDBDE8F3812DE9F8430400DE
S31501A04A500D0000208146002006004A480068B0F1FA
S31501A04A60D17F01D201200600F6B2002E75D1002019
S31501A04A7007003800290080B289B2884207D2BFB2A6
S31501A04A80E05D4049BFB2394408737F1CF1E7ADB27E
S31501A04A903C4885603B4881683B48FEF776FA394831
S31501A04AA0006801F0DBFA804636485FFA88F8404490
S31501A04AB090F8F600002812D134485FFA88F850F829
S31501A04AC0280001F0D1FA002807D101202D495FFA6B
S31501A04AD088F8414481F8F60001E001200600F6B20B
S31501A04AE0002E23D127480068264989680818401E48
S31501A04AF001F0B4FA804623485FFA88F8404490F85A
S31501A04B00F600002812D121485FFA88F850F828004B
S31501A04B1001F0AAFA002807D101201A495FFA88F8FC
S31501A04B20414481F8F60001E001200600F6B2002E0C
S31501A04B3013D11448826892B213491248006801F051
S31501A04B40FFFA002802D00120060006E00D48006801
S31501A04B500C49896808180B4908603000C0B2BDE845
S31501A04B60F2830000743F00008440000017F1DA18B8
S31501A04B70EC3D0000A6540000F53D00009140000068
S31501A04B80F43D0000B0410000BC410000C4A2A00158
S31501A04B90F8B504000D00160000273200290089B2DD
S31501A04BA02000FDF79AFEFFB2002F02D103F062FEAC
S31501A04BB00700FFB2002F02D10020C0B20700FFB24A
S31501A04BC0002F02D103F077FE0700FFB2002F01D11B
S31501A04BD000F003F8FDF79CFEF1BD1CB500208DF891
S31501A04BE00400002004009DF80400002840F08980FC
S31501A04BF044484078012862D19DF8040000280ED1CE
S31501A04C004148007802280AD024208DF8040001A882
S31501A04C10009001233D4A01213720FDF740FC9DF874
S31501A04C20040000280ED13A48007801280AD0702045
S31501A04C308DF8040001A800900123344A01213720F0
S31501A04C40FDF72DFC9DF80400002812D12E48D0F8BE
S31501A04C500C012D49D1F8101188420AD024208DF8D3
S31501A04C60040001A800900123284A01213720FDF75D
S31501A04C7016FC9DF80400002843D12348B0F808117A
S31501A04C802448FFF7E2FE0400E4B2002C0BD1002079
S31501A04C901D4908702048009000231C4A0021372096
S31501A04CA0FDF7FDFB2DE072208DF8040001A8009010
S31501A04CB00123164A01213720FDF7F1FB21E09DF8DA
S31501A04CC0040000280ED10F48007802280AD024201B
S31501A04CD08DF8040001A8009001230C4A0121372078
S31501A04CE0FDF7DDFB9DF8040000280AD10020054947
S31501A04CF00870094800900023044A00213720FDF7D7
S31501A04D00CEFB13BD743F00008440000017F1DA18F2
S31501A04D10A654000091400000F43D0000F8B504003F
S31501A04D200D00160000273200290089B22000FDF7E8
S31501A04D30D4FDFFB2002F02D10020C0B20700FFB2FE
S31501A04D40002F02D103F0D8FD0700FFB2002F02D138
S31501A04D500020C0B20700FFB2002F02D103F0ECFD84
S31501A04D600700FFB2002F02D10020C0B20700FFB298
S31501A04D70002F02D103F0FBFD0700FFB2002F02D1E5
S31501A04D8003F010FE0700FFB2002F01D100F003F8D7
S31501A04D90FDF7BEFDF1BD10B50024E4B2002C02D191
S31501A04DA003F02CFE0400E4B2002C02D103F060FE55
S31501A04DB00400E4B2002C02D10020C0B20400E4B287
S31501A04DC0002C02D10020C0B20400E4B2002C02D112
S31501A04DD003F076FE0400E4B2002C02D10020C0B29A
S31501A04DE00400E4B2002C02D10020C0B20400E4B257
S31501A04DF0002C0FD11948007A10F07F00C0B201280B
S31501A04E0002D0022803D005E000F005F802E000F088
S31501A04E1013F8FFE710BD80B51048007AC0B2C009EB
S31501A04E20C0B2002807D10E48009001230D4A0021E7
S31501A04E308520FDF734FB01BD80B50848007AC0B2D4
S31501A04E40C009C0B2002807D1054800900123054A30
S31501A04E5000218520FDF723FB01BD0000EC3D0000EC
S31501A04E60F43D000017F1DA181224CFE71228DFE784
S31501A04E70010080E0033010E20400000A031051E0B3
S31501A04E801000003A833FB0E101206045B2206021C5
S31501A04E900230A0E110402DE902C0A0E102E0A0E1AC
S31501A04EA0101051E20C502029FCFFFF8A811EB0E1AF
S31501A04EB00C002029042020450111B0E1B220602177
S31501A04EC0012060451080BDE8031091E00120601526
S31501A04ED0020011E3012060151EFF2FE12DE9F0412B
S31501A04EE00020804600200500DFF85803DFF858139C
S31501A04EF008600020DFF854130870DFF84803DFF8D4
S31501A04F00481308600020DFF8481308704FF480604A
S31501A04F1060F30E08022060F31D78FCF7B0E872B6C4
S31501A04F2028F04048DFF82C13C1F80080012161F375
S31501A04F309F78DFF82013C1F80080022161F39F78E2
S31501A04F40DFF81013C1F8008058F04048DFF80413C9
S31501A04F50C1F800800021DFF800231160FCF792E878
S31501A04F60DFF8F8120E0000210F00BFB2042F29D2DC
S31501A04F70301D60F30E08022060F31D78FCF77EE871
S31501A04F8072B628F04048DFF8CC12C1F800800121A2
S31501A04F9061F39F78DFF8BC12C1F80080022161F3AA
S31501A04FA09F78DFF8B012C1F8008058F04048DFF8CA
S31501A04FB0A412C1F8008000217160FCF764E80836EC
S31501A04FC07F1CD2E700200700BFB25E2F36D2DFF8E2
S31501A04FD09002DFF89012BFB2062202FB07F2895AAD
S31501A04FE000EB4100040064F30E05012060F31D757A
S31501A04FF0FCF744E872B625F04045DFF86C120D6067
S31501A05000012161F39F75DFF860120D60022161F342
S31501A050109F75DFF854120D6055F04045DFF8481230
S31501A050200D60DFF84012BFB2062202FB07F211445F
S31501A0503049882180FCF726E87F1CC5E7DFF81C021A
S31501A05040060000200700BFB2042F34D2DFF81C02ED
S31501A05050BFB23901084440683060301D60F30E08C4
S31501A05060022060F31D78FCF70AE872B628F04048E2
S31501A05070DFF8E011C1F80080012161F39F78DFF824
S31501A05080D411C1F80080022161F39F78DFF8C41121
S31501A05090C1F8008058F04048DFF8B811C1F8008087
S31501A050A0DFF8C811BFB23A0189587160FBF7EAEF80
S31501A050B008367F1CC7E74FF4806060F30E08022014
S31501A050C060F31D78FBF7DAEF72B628F04048DFF8F7
S31501A050D08411C1F80080012161F39F78DFF8741172
S31501A050E0C1F80080022161F39F78DFF86811C1F849
S31501A050F0008058F04048DFF85C11C1F8008001211A
S31501A05100DFF854211160FBF7BEEF00210F00BFB2FB
S31501A05110102F07D20020DFF85811BFB241F827009F
S31501A051207F1CF4E71F220FF258111820FCF72AF86A
S31501A051301F220FF280111920FCF724F81F220FF26B
S31501A05140A8111A20FCF71EF81F220FF2D0111B205E
S31501A05150FCF718F81F220FF2F8111C20FCF712F821
S31501A051601F220FF220211D20FCF70CF81F220FF29F
S31501A0517048211E20FCF706F81F220FF270211F20DE
S31501A05180FCF700F81F220FF298212020FBF7FAFF67
S31501A051901F220FF2C0212120FBF7F4FF1F220FF2DD
S31501A051A0E8212220FBF7EEFF1F220FF21031232068
S31501A051B0FBF7E8FF1F220FF238312420FBF7E2FFAD
S31501A051C01F220FF260312520FBF7DCFF1F220FF211
S31501A051D088312620FBF7D6FF1F220FF2B0312720F8
S31501A051E0FBF7D0FFBDE8F08138B50400E4B2102C7E
S31501A051F025D25FF00110A04020F07F4005001E4897
S31501A0520005601D480068BFF35F8F1A4805601948FD
S31501A05210006800BF00BF00BF00BF00BF00BF1448A9
S31501A05220E4B250F82400002804D01148E4B250F8A2
S31501A0523024008047E4B214F118001049086031BD7A
S31501A052400000000055CEAC5C000060B0153480B003
S31501A05250163480B0048473B4008473B4008273B42A
S31501A05260000074B4409EA001000474B4A0A5A001DE
S31501A05270943D0000080062B0100062B0480C40B036
S31501A0528004E04EE20F502DE9100AF1EE01002DE9DE
S31501A0529004D04DE2100B2DED0000A0E3D1FFFFFAE3
S31501A052A0100BBDEC04D08DE20100BDE8100AE1EEC1
S31501A052B00F90FDE804E04EE20F502DE9100AF1EE41
S31501A052C001002DE904D04DE2100B2DED0100A0E364
S31501A052D0C4FFFFFA100BBDEC04D08DE20100BDE8BE
S31501A052E0100AE1EE0F90FDE804E04EE20F502DE921
S31501A052F0100AF1EE01002DE904D04DE2100B2DEDBF
S31501A053000200A0E3B7FFFFFA100BBDEC04D08DE2BB
S31501A053100100BDE8100AE1EE0F90FDE804E04EE2BF
S31501A053200F502DE9100AF1EE01002DE904D04DE24E
S31501A05330100B2DED0300A0E3AAFFFFFA100BBDECA5
S31501A0534004D08DE20100BDE8100AE1EE0F90FDE860
S31501A0535004E04EE20F502DE9100AF1EE01002DE90D
S31501A0536004D04DE2100B2DED0400A0E39DFFFFFA42
S31501A05370100BBDEC04D08DE20100BDE8100AE1EEF0
S31501A053800F90FDE804E04EE20F502DE9100AF1EE70
S31501A0539001002DE904D04DE2100B2DED0500A0E38F
S31501A053A090FFFFFA100BBDEC04D08DE20100BDE821
S31501A053B0100AE1EE0F90FDE804E04EE20F502DE950
S31501A053C0100AF1EE01002DE904D04DE2100B2DEDEE
S31501A053D00600A0E383FFFFFA100BBDEC04D08DE21B
S31501A053E00100BDE8100AE1EE0F90FDE804E04EE2EF
S31501A053F00F502DE9100AF1EE01002DE904D04DE27E
S31501A05400100B2DED0700A0E376FFFFFA100BBDEC04
S31501A0541004D08DE20100BDE8100AE1EE0F90FDE88F
S31501A0542004E04EE20F502DE9100AF1EE01002DE93C
S31501A0543004D04DE2100B2DED0800A0E369FFFFFAA1
S31501A05440100BBDEC04D08DE20100BDE8100AE1EE1F
S31501A054500F90FDE804E04EE20F502DE9100AF1EE9F
S31501A0546001002DE904D04DE2100B2DED0900A0E3BA
S31501A054705CFFFFFA100BBDEC04D08DE20100BDE884
S31501A05480100AE1EE0F90FDE804E04EE20F502DE97F
S31501A05490100AF1EE01002DE904D04DE2100B2DED1D
S31501A054A00A00A0E34FFFFFFA100BBDEC04D08DE27A
S31501A054B00100BDE8100AE1EE0F90FDE804E04EE21E
S31501A054C00F502DE9100AF1EE01002DE904D04DE2AD
S31501A054D0100B2DED0B00A0E342FFFFFA100BBDEC64
S31501A054E004D08DE20100BDE8100AE1EE0F90FDE8BF
S31501A054F004E04EE20F502DE9100AF1EE01002DE96C
S31501A0550004D04DE2100B2DED0C00A0E335FFFFFA00
S31501A05510100BBDEC04D08DE20100BDE8100AE1EE4E
S31501A055200F90FDE804E04EE20F502DE9100AF1EECE
S31501A0553001002DE904D04DE2100B2DED0D00A0E3E5
S31501A0554028FFFFFA100BBDEC04D08DE20100BDE8E7
S31501A05550100AE1EE0F90FDE804E04EE20F502DE9AE
S31501A05560100AF1EE01002DE904D04DE2100B2DED4C
S31501A055700E00A0E31BFFFFFA100BBDEC04D08DE2D9
S31501A055800100BDE8100AE1EE0F90FDE804E04EE24D
S31501A055900F502DE9100AF1EE01002DE904D04DE2DC
S31501A055A0100B2DED0F00A0E30EFFFFFA100BBDECC3
S31501A055B004D08DE20100BDE8100AE1EE0F90FDE8EE
S31501A055C000208149086028207F4948604FF4FA608D
S31501A055D07D49886000207D49088000207C4908809B
S31501A055E07C487D49086003207C49086079487A494E
S31501A055F008607B487B4908607648774908600120A6
S31501A056007949086079480078C0B20028FAD1714872
S31501A0561071490860012076490860704780B51F224C
S31501A056200FF24001DA20FBF7ADFD01BD69486A49D9
S31501A05630086007206C490860664867490860002031
S31501A056406B4908606348644908600120694908609C
S31501A0565066480078C0B20028FAD170475C48008835
S31501A056607047000004E04EE21F502DE9100AF1EE4A
S31501A0567001002DE9100B2DED6A0D00FA44019FE5FD
S31501A05680000090E5010090E238119FE5000081E558
S31501A0569030019FE5000090E528119FE5041091E5F2
S31501A056A0010050E10A00003A20019FE5B000D0E1D7
S31501A056B00040B0E1020094E210119FE5B000C1E103
S31501A056C000019FE5000090E5280090E2F4109FE517
S31501A056D0040081E5EC009FE5000090E5E4109FE55C
S31501A056E0081091E5010050E10500003A4F0D00FABE
S31501A056F0D0009FE5000090E57D0E90E2C4109FE5E5
S31501A05700080081E5BC009FE5000090E52008B0E116
S31501A057100008B0E1000050E31100000AA4009FE5D3
S31501A05720B000D0E10008B0E12008B0E194109FE5F7
S31501A05730000081E58C009FE5B400D0E10008B0E14E
S31501A057402008B0E17C109FE5040081E574009FE587
S31501A05750B800D0E10008B0E12008B0E164109FE5EF
S31501A05760080081E55C009FE5000090E558109FE5E3
S31501A05770B000C1E100000FE180000CF150109FE5DF
S31501A05780B024A0E3602882E3001082E50110A0E323
S31501A0579060209FE50010C2E500100FE1C010C1E333
S31501A057A0C00000E2001081E101F021E1DA10A0E3DE
S31501A057B044209FE5001082E5100BBDEC0100BDE879
S31501A057C0100AE1EE1F90FDE8DC3D00009C540000AC
S31501A057D09E54000055CEAC5C000060B0040560B0DC
S31501A057E032000300080560B0000560B0622880B0F1
S31501A057F0100560B0140560B0A02880B0480C40B078
S31501A0580080B5DFF83806DFF8381608600020DFF823
S31501A0581034160870DFF82406DFF82416086007207E
S31501A05820DFF824160860DFF81406DFF814160860FE
S31501A058300020DFF818160860DFF80006DFF800166A
S31501A0584008600120DFF808160860DFF8080600786E
S31501A05850C0B20028F9D1DFF8E405DFF8E415086045
S31501A058605FF08060DFF8F0150860DFF8D005DFF89B
S31501A05870D01508600220DFF8E4150860DFF8BC0542
S31501A05880DFF8BC150860DFF8D805DFF8D815086081
S31501A05890DFF8A805DFF8A81508600120DFF8A8152C
S31501A058A00860DFF89805DFF898150860FF20DFF893
S31501A058B0B8150860DFF88405DFF884150860DFF8FD
S31501A058C0AC05DFF8AC150860DFF87005DFF87015D8
S31501A058D00860DFF8A005DFF8A0150860DFF85C0511
S31501A058E0DFF85C150860DFF89405DFF89415086009
S31501A058F0DFF84805DFF848150860DFF88805DFF806
S31501A0590088150860DFF83405DFF834150860DFF87C
S31501A059107C05DFF87C150860DFF82005DFF8201587
S31501A059200860DFF86005DFF86C150860DFF80C0584
S31501A05930DFF80C1508602920DFF85C150860DFF890
S31501A05940FC04DFF8FC140860DFF84005DFF84C150D
S31501A059500860DFF8E804DFF8E81408600520DFF83E
S31501A0596040150860DFF8D404DFF838150860052073
S31501A05970DFF834150860DFF8C404DFF828150860DD
S31501A059800020DFF828150860DFF8B004DFF8141549
S31501A0599008604FF48060DFF818150860DFF89C04F2
S31501A059A0DFF800150860DFF80C05DFF80C150860B4
S31501A059B0DFF88804DFF8EC1408600020DFF8FC1497
S31501A059C00860DFF87804DFF8DC1408600020DFF84F
S31501A059D0F0140860DFF86404DFF86414086003209B
S31501A059E0DFF8E0140860DFF85404DFF8B8140860A3
S31501A059F0DFF8D404DFF8D4140860DFF84004DFF838
S31501A05A00A41408603020DFF8C8140860DFF82C045D
S31501A05A10DFF890140860DFF8BC04DFF8BC14086056
S31501A05A20DFF81804DFF87C140860DFF8B004DFF8AB
S31501A05A30B0140860DFF80404DFF8681408600020D9
S31501A05A40DFF8A0140860DFF8F403DFF85814086043
S31501A05A500020DFF894140860DFF8E003DFF84414AF
S31501A05A6008600020DFF884140860DFF8D003DFF8AF
S31501A05A70341408600020DFF878140860DFF8BC034E
S31501A05A80DFF8201408600020DFF868140860DFF84A
S31501A05A90AC03DFF8101408600020DFF85C1408607E
S31501A05AA001F072FADFF89403DFF8F8130860AB206F
S31501A05AB0DFF848140870DFF88403DFF88413086060
S31501A05AC0AB20DFF83C140860DFF838040078C0B2D8
S31501A05AD00028F9D0DFF86403DFF864130860012019
S31501A05AE0DFF824140870DFF8A8030068C0F381105A
S31501A05AF0002808D1DFF84403DFF844130860012029
S31501A05B00DFF808140870DFF894030068C0F3811069
S31501A05B10002808D1DFF82403DFF824130860012048
S31501A05B20DFF8EC130870DFF868030068C0F3811092
S31501A05B300228F8D1DFF864030068C0F381100228B7
S31501A05B40F8D1DFF8D0030078C0B200280ED0DFF874
S31501A05B50EC02DFF8EC1208600020DFF8BC13086045
S31501A05B60DFF8B803DFF8B813086010E0DFF8B40374
S31501A05B700068DFF8B413884205D1DFF8AC03DFF87B
S31501A05B80A013086003E00020DFF89413086000204A
S31501A05B90DFF89013086001BD80B5A848A849086040
S31501A05BA0DFF88803DFF870130860DFF8F0020068F9
S31501A05BB0C0F38110022806D1A048A149086001209E
S31501A05BC0DFF84C130870B2480068C0F381100228B0
S31501A05BD006D19A489A4908600120DFF83013087067
S31501A05BE0AB480068C0F381100028F9D1AB48006822
S31501A05BF0C0F381100028F9D1904891490860072087
S31501A05C009F4908608D488E4908600020A449086014
S31501A05C108A48A44908600020A34908608748A14989
S31501A05C2008600020A149086084489E4908600020B8
S31501A05C309F49086081489B4908600020A3490860E4
S31501A05C407E487F49086000209E4908607B489549A7
S31501A05C500860AB20A9490870784879490860AB204B
S31501A05C60A7490860A7480078C0B20028FAD001F079
S31501A05C708BF97248724908600120A34908706F48E0
S31501A05C806F4908605FF00440734908606B486C492E
S31501A05C9008605FF44030A649086068486849086012
S31501A05CA00620A44908606548654908600720A249FD
S31501A05CB008606248624908600020A04908605F4800
S31501A05CC05F49086000209E4908605C485C490860FD
S31501A05CD066489C49086059485949086000209A4974
S31501A05CE0086056485649086080209849086053487C
S31501A05CF06C49086096489749086050486949086008
S31501A05D005FF00130944908604C486649086040F24A
S31501A05D1001109249086049486249086000209049EB
S31501A05D20086046485F49086000208E4908604348DC
S31501A05D305C49086000208C490860404859490860C0
S31501A05D4000208A4908603D485649086000208849D4
S31501A05D5008603A48534908600020864908603748D8
S31501A05D605049086000208449086034484D490860BC
S31501A05D7000208249086031484A49086000208049CC
S31501A05D8008602E484749086000207E4908602B48D4
S31501A05D904449086000207C490860284841490860B8
S31501A05DA000207A49086025483E49086000207849C4
S31501A05DB008602248224908600120764908701F48D8
S31501A05DC038490860BA20744908701C481C49086003
S31501A05DD0BA201C49087071480078C0B20128FAD0CF
S31501A05DE001F0D2F8BFF34F8FBFF36F8F30BF4E488C
S31501A05DF04C49086000BF00BF00BF00BF00BF00BF85
S31501A05E0000BF00BF72B60D480D490860A5206449C0
S31501A05E10087001BD42490968404A914202D1012157
S31501A05E20080009E03E4909683F4A914202D1022190
S31501A05E30080001E000210800C0B2704755CEAC5C55
S31501A05E40000060B07C0160B0000560B0100560B0D4
S31501A05E50140560B0622880B0040660B0040560B085
S31501A05E6000020600080560B00C0660B0000F000134
S31501A05E70C40060B000010300800060B00F01010002
S31501A05E80840060B000012100940060B001480400C4
S31501A05E90100660B0A40060B0A80060B0200660B093
S31501A05EA0880060B0000030B0800030B0840030B00F
S31501A05EB0880030B0F14FBFFF8C0030B0900030B0F9
S31501A05EC0940030B0900060B000110103980030B08A
S31501A05ED09C0030B031030101A00030B003030101E1
S31501A05EE0A40030B0A80030B0AC0030B0B00030B0E3
S31501A05EF0B40030B0B80030B0BC0030B0FC0030B057
S31501A05F00FC0060B0441480B0841480B0813080B0AD
S31501A05F10013180B0183480B0800660B05CA3A35C68
S31501A05F2004000002080000025A96A56900020001B9
S31501A05F30000160B0040160B0080160B00C0160B05E
S31501A05F40100160B0440160B0480160B04C0160B07E
S31501A05F5001000001000130B0040130B0080130B0E9
S31501A05F600C0130B0100130B0140130B0180130B0BE
S31501A05F701C0130B0200130B0240130B0280130B06E
S31501A05F802C0130B0300130B0340130B0380130B01E
S31501A05F903C0130B0851480B07C0130B0471480B08C
S31501A05FA0820360B029480068294943F2390201FBFE
S31501A05FB0002026490860704780B526488068234995
S31501A05FC0086024488079032803D22248007903284F
S31501A05FD001D300F036F801BD80B51F4840780128ED
S31501A05FE02ED11D4840884FF6F071884228D21A4812
S31501A05FF04088401C1849488017484088B0F5FA7F68
S31501A060001ED114480079032802D302201149087130
S31501A0601010488079032802D302200E4988710020F6
S31501A060200D49087000200C49488000200A49487093
S31501A0603000F0A6F90123032206490220FCF747FE38
S31501A0604001BD01200449487070470000A03A000034
S31501A060506D4EC641003F0000F03E0000B0F1D07089
S31501A06060C00BC0B270470000F8B50400002772B695
S31501A06070BFF34F8FBFF36F8FDFF84C030078C0B229
S31501A06080002810D002F0B0FF0500EDB2002DF9D125
S31501A0609000200700BFB2B7F5FA7F04D200BF00F017
S31501A060A073FF7F1CF6E700200700BFB2B7F5FA7FA2
S31501A060B004D200BF00F068FF7F1CF6E7C248007853
S31501A060C0C0B2002823D102F06FFF0500EDB2002D6A
S31501A060D0F9D100200700BFB2B7F5FA7F04D200BFFD
S31501A060E000F052FF7F1CF6E70121200002F0A4FD7B
S31501A060F000200700BFB2B7F5FA7F04D200BF00F0B7
S31501A0610043FF7F1CF6E762B60020060002E062B6F6
S31501A061100120060000200700BFB2B7F5FA7F04D21E
S31501A0612000BF00F031FF7F1CF6E73000C0B2F2BD20
S31501A0613010B504000121200002F054FE10BD00009C
S31501A061402DE9FE4F04000D00160000275FF00008A0
S31501A061505FF0000968469D49D1E90023C0E9002303
S31501A0616072B6BFF34F8FBFF36F8F97480078C0B257
S31501A06170002811D102F018FF82465FFA8AFABAF115
S31501A06180000FF7D100200700BFB2FF2F04D200BF36
S31501A0619000F0FAFE7F1CF7E700200700BFB2B6B2F7
S31501A061A0B6B216F00300301A874212D200BF00BF62
S31501A061B000BF00BFBFB2E859029014FA87F0834628
S31501A061C00122BFB2E95914FA87F002F09DFD3F1DE5
S31501A061D0E4E700200700BFB2FF2F04D200BF00F002
S31501A061E0D3FE7F1CF7E703210E4231D00020804663
S31501A061F01FFA88F8B8F1080F08D2FF2069461FFADE
S31501A0620088F801F8080018F10108F1E716F0030073
S31501A06210804616F00300301A070000208146484642
S31501A06220414680B289B288420CD21FFA89F919FA7D
S31501A0623087F0285C69461FFA89F901F8090019F166
S31501A062400109ECE70122009914FA87F002F05CFD3E
S31501A0625062B60020BDE8FE8F30B5F3B068464FF4B4
S31501A06260E47102F0EEEE72B6BFF34F8FBFF36F8FFC
S31501A0627055480078C0B200280FD002F0B5FE05003F
S31501A06280EDB2002DF9D100200400E4B2FF2C04D018
S31501A0629000BF00F079FE641CF7E74B480078C0B256
S31501A062A0002869D1012000900120019001200290CF
S31501A062B003208DF80C0010208DF81C0000208DF80D
S31501A062C01D005FF0D17006900120099003208DF882
S31501A062D0280011208DF8380000208DF839005FF0D4
S31501A062E0D2700D900120109003208DF84400122049
S31501A062F08DF8540000208DF855005FF0D4701490ED
S31501A063000120179003208DF8600012208DF87000EF
S31501A0631000208DF871005FF0D8701B9001201E90AF
S31501A0632003208DF87C0012208DF88C0000208DF8BA
S31501A063308D005FF0DC7022900120259003208DF85E
S31501A06340980015208DF8A80001208DF8A9005FF00E
S31501A063506060299001208DF8A10001208DF89F0091
S31501A0636001208DF8A000684602F06EFE02F01CFE28
S31501A063700500EDB2002DF9D162B673B030BD0000B3
S31501A0638038B500200500ADB2B5F5FA7F04D200BF3D
S31501A0639000F0FAFD6D1CF6E70B480078C0B20028A4
S31501A063A010D002F021FE0400E4B2002CF9D10020A5
S31501A063B00500ADB2B5F5FA7F04D200BF00F0E4FD49
S31501A063C06D1CF6E731BD0000448018B16CA7A00191
S31501A063D080B50020DFF8081B08700020DFF8001B3D
S31501A063E048800020DFF8F81A88800020DFF8F01A2C
S31501A063F088600020DFF8E81AC8601F220FF608217E
S31501A064001420FAF7BFFE01BDDFF8D40A0078704761
S31501A064102DE9F04F83B000208DF8040000208146BD
S31501A064205FFA89F9B9F10E0F68D2DFF8B80A5FFAF7
S31501A0643089F910F83900DFF8B01A5FFA89F95FEA2D
S31501A0644009128854DFF8A00A5FFA89F95FEA0911EF
S31501A06450405C00284FD001208DF804000020DFF811
S31501A06460881A5FFA89F95FEA091211444870002077
S31501A06470DFF8741A5FFA89F95FEA091211444880B4
S31501A064800020DFF8641A5FFA89F95FEA091211445C
S31501A064908880DFF8500A5FFA89F900EBC9004088C5
S31501A064A0DFF8441A5FFA89F95FEA091211440881F3
S31501A064B04FF48050DFF8301A5FFA89F95FEA0912C2
S31501A064C011440989B0FBF1F0DFF81C1A5FFA89F9CA
S31501A064D05FEA09121144C880DFF8080A5FFA89F950
S31501A064E000EBC9004068DFF8001A5FFA89F95FEA94
S31501A064F009121144C86019F1010991E79DF8040038
S31501A06500002800F02A81002081465FFA89F9B9F1B5
S31501A065100E0F80F02281DFF8D0095FFA89F95FEAD0
S31501A065200911405C002800F015810120DFF8B81997
S31501A065305FFA89F95FEA091288545FFA89F94FF47B
S31501A06540005000FB09F010F16060804600208246F1
S31501A0655000208DF8050001200500EDB2002D5ED0CA
S31501A065601FFA8AFADFF880095FFA89F95FEA091149
S31501A065700844008900FB0A80070038680090BDF82E
S31501A065800000BDF8021011FA80F04FF6FF718842A3
S31501A065902FD10020050001208DF8050001208DF8DE
S31501A065A004000220DFF840195FFA89F95FEA0912AF
S31501A065B088540020DFF830195FFA89F95FEA0912D9
S31501A065C011444870DFF820095FFA89F95FEA0911D9
S31501A065D00844A0F804A0BDF80000DFF80C195FFA82
S31501A065E089F95FEA091211444880BDF80000060046
S31501A065F0B3E71AF1010A5046DFF8EC185FFA89F9F8
S31501A066005FEA09121144C98880B28842A5D31FFA4C
S31501A066108AFABAF1030FA0D3002005009DE718F569
S31501A0662080580020824601200500EDB2002D00F021
S31501A0663091801FFA8AFADFF8B0085FFA89F95FEA52
S31501A0664009110844008900FB0A80070038680090F8
S31501A06650BDF80000BDF8021011FA80F04FF6FF71E7
S31501A0666088425FD10020050001208DF804009DF825
S31501A06670050000282AD101208DF805000220DFF8A7
S31501A0668068185FFA89F95FEA091288540120DFF8D0
S31501A0669058185FFA89F95FEA091211444870DFF8C0
S31501A066A048085FFA89F95FEA09110844A0F804A02D
S31501A066B0BDF80000DFF830185FFA89F95FEA091220
S31501A066C011444880BDF800000600AEE7BDF8000001
S31501A066D0B6B2801BDFF810185FFA89F95FEA0912D2
S31501A066E01144C988C91C88429FD20120DFF8F81736
S31501A066F05FFA89F95FEA091211444870DFF8E807E1
S31501A067005FFA89F95FEA09110844A0F804A0BDF867
S31501A067100000DFF8D4175FFA89F95FEA091211447C
S31501A06720488082E71AF1010A5046DFF8BC175FFAE2
S31501A0673089F95FEA09121144C98880B28842FFF437
S31501A0674074AF1FFA8AFABAF1030FFFF46EAF0020F5
S31501A0675005006AE719F10109D7E69DF804000028AA
S31501A0676000F05781002081465FFA89F9B9F10E0F31
S31501A0677080F04F81DFF870075FFA89F95FEA0911A6
S31501A06780405C022840F042815FFA89F94FF400503B
S31501A06790DFF854175FFA89F95FEA091211444978BB
S31501A067A04FF48052514300FB091010F160608046FE
S31501A067B0DFF834075FFA89F95FEA091108444088CE
S31501A067C08346DFF824075FFA89F95FEA09110844CD
S31501A067D08088824601200500EDB2002D53D01AF122
S31501A067E0010A1BF1010B5046DFF8FC165FFA89F985
S31501A067F05FEA09121144C98880B288420DD21FFAF4
S31501A068008AFADFF8E4065FFA89F95FEA0911084412
S31501A068108088BAEB0000032802D300200500DBE73D
S31501A068201FFA8AFADFF8C0065FFA89F95FEA091149
S31501A068300844008900FB0A80070038680090BDF86B
S31501A068400000BDF8021011FA80F04FF6FF718842E0
S31501A06850C2D1BDF80000594689B28842BCD1DFF841
S31501A0686088065FFA89F95FEA09110844A0F804A02D
S31501A06870BDF80000DFF870165FFA89F95FEA091220
S31501A0688011444880A8E7DFF860065FFA89F95FEA54
S31501A068900911084480888246DFF84C065FFA89F917
S31501A068A05FEA09110844408883465E460120050037
S31501A068B001220121002002F00FFD1FFA8AFADFF85A
S31501A068C028065FFA89F95FEA09110844008900FBE5
S31501A068D00A80070038680090BDF80000BDF80210D4
S31501A068E011FA80F04FF6FF71884253D15846BDF890
S31501A068F0001080B288424DD15E46DFF8EC055FFA02
S31501A0690089F95FEA0911084400898008401EADF89B
S31501A069100600002004002000BDF8061080B28842BF
S31501A069201BD2DFF8C4055FFA89F95FEA09110844A9
S31501A06930C068A4B2396840F82410DFF8AC055FFA44
S31501A0694089F95FEA09110844C068A4B250F8240085
S31501A0695002F0DDFC3F1D641CDDE7DFF88C055FFA64
S31501A0696089F95FEA09110844C068A4B2396840F8F8
S31501A06970241002F0CFFCDFF870155FFA89F95FEAFF
S31501A0698009121144C968A4B251F82410814201D157
S31501A0699000200500EDB2002D34D0BBF1010BB6B23B
S31501A069A01FFA8BFBB6EB0B00042821D21FFA8AFA39
S31501A069B0BAF1000F19D1DFF830055FFA89F95FEA5C
S31501A069C009110844C088401E8246DFF81C055FFAFB
S31501A069D089F95FEA091108444078002802D0B8F580
S31501A069E080580FE018F580580CE0BAF1010A09E0C9
S31501A069F0002005000320DFF8F0145FFA89F95FEAA9
S31501A06A0009128854EDB2002D7FF452AF19F1010994
S31501A06A10AAE6BDE8F78F0100C9B20E2906D2DFF8B2
S31501A06A20C824C9B20B01D25C100001E000221000FB
S31501A06A30C0B2704770B40300DBB20E2B33D200296B
S31501A06A4031D092B2002A2ED0DFF89C54DBB21E01BF
S31501A06A5035442D89083DAD0892B2954220D3DFF881
S31501A06A608854DBB21E01AD5D022D19D100252C0083
S31501A06A7025001600ADB2B6B2B5420ED2DFF8685403
S31501A06A80DBB21E013544ED68A4B205EB84056D6841
S31501A06A90A4B241F82450641CEAE70025280004E0CA
S31501A06AA00125280001E001252800C0B270BC70476D
S31501A06AB02DE9F04F83B004000D009146E4B20E2CEF
S31501A06AC080F09C81002D00F099811FFA89F9B9F116
S31501A06AD0000F00F09381DFF808040078002840F049
S31501A06AE08D81DFF80404E4B2210108440089083845
S31501A06AF080081FFA89F94845C0F07D81DFF8E803CF
S31501A06B00E4B22101405C002800F0758100208DF8D7
S31501A06B100400DFF8D403E4B2210108440089800807
S31501A06B20401E060001220121002002F0D5FBDFF85C
S31501A06B30B803E4B22101405C022858D1DFF8A803CA
S31501A06B40E4B2210108448088401CDFF89C13E4B21A
S31501A06B50220111448880DFF89003E4B221010844A0
S31501A06B608088DFF88413E4B222011144C9888842DF
S31501A06B701CD301208DF804000020DB49E4B22201D8
S31501A06B8011448880D848E4B22101084440780028FD
S31501A06B9006D10120D449E4B222011144487005E08E
S31501A06BA00020D149E4B2220111444870CE48E4B292
S31501A06BB0210108444088401CCB49E4B2220111447A
S31501A06BC04880C948E4B2210108444088ADF80000D4
S31501A06BD04FF6FF70BDF80010401AADF802000098FC
S31501A06BE0C149E4B222011144C968086030E001201C
S31501A06BF08DF804000020BC49E4B22201114488802A
S31501A06C000020B949E4B22201114448700020B649D6
S31501A06C10E4B2220111444880B448B349E4B2220146
S31501A06C201144C9680860012082465046310080B2ED
S31501A06C3089B288420CD2AC48E4B221010844C068AA
S31501A06C401FFA8AFA002140F82A101AF1010AECE784
S31501A06C50A548E4B221010844C068006802F057FBC8
S31501A06C6019F10109012082465046494680B289B2EE
S31501A06C7088421CD29C48E4B221010844C0681FFA8C
S31501A06C808AFA1FFA8AFA05EB8A0151F8041C40F820
S31501A06C902A109548E4B221010844C0681FFA8AFA6D
S31501A06CA050F82A0002F033FB1AF1010ADCE750463C
S31501A06CB0310080B289B288420DD28B48E4B221015B
S31501A06CC00844C0681FFA8AFA50F82A0002F01FFB8E
S31501A06CD01AF1010AEBE702F01DFB8349E4B2220196
S31501A06CE01144C9681FFA8AFA41F82A00E4B24FF49E
S31501A06CF0005000FB04F010F1606083467A48E4B2CC
S31501A06D002101084440784FF4805101FB00BB76482D
S31501A06D10E4B22101084400897349E4B22201114475
S31501A06D20898801FB00BBFAF7AAE972B6704909780E
S31501A06D30C9B2002908D06F496F4A116001216F4A73
S31501A06D4011700021884601E001218846FAF79AE9E7
S31501A06D506B490978C9B2002901D1012080465FFAA1
S31501A06D6088F8B8F1000F4BD101205D4908705E4843
S31501A06D70E4B22101084400898008594988805A480B
S31501A06D80E4B221010844C0685549C86001205D49A3
S31501A06D90087001205C4908709DF80400002818D0ED
S31501A06DA000204F4948804E48C0F808B0002007008F
S31501A06DB0022060F30307E4B260004B49E4B222016A
S31501A06DC01144497850FA81F060F317474F4807609C
S31501A06DD00BE00120424948801BF10400404988602C
S31501A06DE03F48C0680068CBF8000002203E49E4B2E3
S31501A06DF02201885404E00120804601E0012080465A
S31501A06E004046C0B2BDE8FE8F07002DE90100A0E310
S31501A06E10EC109FE50000C1E5C0009FE5B200D0E1FE
S31501A06E20B8109FE5B410D1E1010050E11300002A8A
S31501A06E30A8009FE50C0090E5A0109FE5B210D1E156
S31501A06E400111B0E1010090E790109FE5081091E5CE
S31501A06E50000081E584009FE5B200D0E1010090E247
S31501A06E6078109FE5B200C1E170009FE5080090E5AA
S31501A06E70040090E264109FE5080081E5120000EA93
S31501A06E800000A0E354109FE50000C1E50000A0E3C7
S31501A06E9070109FE50000C1E500000FE180000CF134
S31501A06EA04C109FE54C209FE5001082E50010A0E361
S31501A06EB044209FE50010C2E500100FE1C010C1E318
S31501A06EC0C00000E2001081E101F021E11400A0E37D
S31501A06ED038109FE5000081E50700BDE804F05EE2F9
S31501A06EE088540000F0A4A001A85300000000FFFFF1
S31501A06EF0580319B1A5F16DCF002041B0480019B1D1
S31501A06F00400119B1280119B1200119B1542041B08C
S31501A06F10480C40B010B5FAF7B2E8040072B63A4888
S31501A06F203A49086001203A4908703748374908604C
S31501A06F300120384908703448344908600020364990
S31501A06F4008603148354908600020354908702E4847
S31501A06F50324908604FF48270324908602A482F49A5
S31501A06F60086001202E4908700F220FF27001062039
S31501A06F70FAF7BFF81F220FF230010220FAF702F941
S31501A06F802000FAF780E810BD00B5FAF778E872B6E6
S31501A06F9025490968254A116025490968254A1160CC
S31501A06FA0FAF770E800BD000003002DE984009FE513
S31501A06FB0B014A0E3601881E3000081E5A500A0E379
S31501A06FC074109FE50000C1E50200A0E36C109FE5E7
S31501A06FD0000081E50300BDE804F05EE254809FE570
S31501A06FE0B094A0E3609889E3008089E5A5A0A0E319
S31501A06FF044B09FE500A0CBE506C0A0E33C809FE599
S31501A0700000C088E504F05EE255CEACED00C060B0EC
S31501A07010200186B0210186B00CC060B0008030B0DE
S31501A07020580204B1488030B02CC060B010C060B026
S31501A0703030C060B018C060B055CEAC5C820360B001
S31501A07040480C40B000B583B000208DF80400A948D3
S31501A07050808800280BD113208DF8040001A8009088
S31501A070600123A54A01211020FBF719FA02E000200D
S31501A070708DF804009DF804000EBD00B583B0002074
S31501A070808DF804009B48808801280BD013208DF829
S31501A07090040001A800900123974A01211020FBF7C3
S31501A070A0FEF902E000208DF804009DF804000EBD53
S31501A070B000B583B000208DF804008E48007A10F048
S31501A070C07F00012812D18B48808800280BD113207C
S31501A070D08DF8040001A800900123874A0121102000
S31501A070E0FBF7DDF902E000208DF804008148007A63
S31501A070F010F07F00022812D17E48808800280BD18B
S31501A0710013208DF8040001A8009001237A4A0121D9
S31501A071101020FBF7C4F902E000208DF804007548A1
S31501A07120007A10F07F00032812D1724880880028C7
S31501A071300BD113208DF8040001A8009001236E4AFB
S31501A0714001211020FBF7ABF902E000208DF8040025
S31501A071509DF804000EBD00B583B000208DF8040093
S31501A071606448007A10F07F0001280BD06148007AAC
S31501A0717010F07F00022805D05E48007A10F07F004B
S31501A07180032803D100208DF804000FE012208DF80A
S31501A071900400584800685949884207D101A80090BF
S31501A071A00123554A01211020FBF779F99DF8040026
S31501A071B00EBD1CB500208DF80400FBF700FD0400F0
S31501A071C04F48844203D100208DF804003BE0494892
S31501A071D0007A10F07F00032817D1FBF77AFB02286B
S31501A071E010D17E208DF804004248006843498842A8
S31501A071F00BD101A8009001233F4A01211020FBF7E2
S31501A072004EF902E000208DF804003A48007A10F009
S31501A072107F00022817D1FBF75CFB012810D17E2045
S31501A072208DF8040033480068344988420BD101A87F
S31501A0723000900123304A01211020FBF730F902E02A
S31501A0724000208DF804009DF8040016BD00B583B09A
S31501A0725000208DF804002748007A10F07F0001284D
S31501A0726012D12448808801280BD013208DF8040060
S31501A0727001A800900123204A01211020FBF70FF954
S31501A0728002E000208DF804001A48007A10F07F0071
S31501A07290022812D11748808801280BD013208DF817
S31501A072A0040001A800900123134A01211020FBF735
S31501A072B0F6F802E000208DF804000E48007A10F0DE
S31501A072C07F00032812D10B48808801280BD01320F8
S31501A072D08DF8040001A800900123074A012110207E
S31501A072E0FBF7DDF802E000208DF804009DF804000C
S31501A072F00EBD0000EC3D000017F1DA18F117DA18FF
S31501A07300A35A7AA700B583B000208DF80400FBF735
S31501A07310E0FA012810D17F208DF804007348006897
S31501A07320734988420BD101A800900123714A01211A
S31501A073301120FBF7B4F802E000208DF804009DF8B7
S31501A0734004000EBD00B583B000208DF80400674887
S31501A07350808800280BD113208DF8040001A8009085
S31501A073600123644A01211120FBF799F802E00020CC
S31501A073708DF804009DF804000EBD00B583B0002071
S31501A073808DF804005948808801280BD013208DF868
S31501A07390040001A800900123564A01211120FBF700
S31501A073A07EF802E000208DF804009DF804000EBDD1
S31501A073B000B583B000208DF804004C48007A10F087
S31501A073C07F00012812D14948808800280BD11320BB
S31501A073D08DF8040001A800900123464A012111203D
S31501A073E0FBF75DF802E000208DF804003F48007A23
S31501A073F010F07F00032812D13C48808800280BD1C9
S31501A0740013208DF8040001A800900123394A012117
S31501A074101120FBF744F802E000208DF804009DF846
S31501A0742004000EBD00B583B000208DF804002F48DE
S31501A07430007A10F07F00012805D02C48007A10F0C0
S31501A074407F00032803D100208DF804000FE012204D
S31501A074508DF80400254800682549884207D101A86E
S31501A0746000900123234A01211120FBF718F89DF86A
S31501A0747004000EBD00B583B000208DF804001B48A2
S31501A07480007A10F07F00012812D1184880880128BF
S31501A074900BD013208DF8040001A800900123154AF2
S31501A074A001211120FAF7FBFF02E000208DF804006C
S31501A074B00E48007A10F07F00032812D10B4880886D
S31501A074C001280BD013208DF8040001A800900123F8
S31501A074D0084A01211120FAF7E2FF02E000208DF807
S31501A074E004009DF804000EBD00000000EC3D000064
S31501A074F0F117DA1817F1DA1800B583B000208DF864
S31501A0750004003C48808802280BD213208DF8040081
S31501A0751001A800900123384A01212220FAF7BFFFD2
S31501A0752002E000208DF804009DF804000EBD1CB5F4
S31501A0753031208DF8040000200400E4B2092C12D2F7
S31501A075402C48007A000280B22A49497A08432B497D
S31501A07550E4B231F81410884203D100208DF804005A
S31501A0756001E0641CE9E79DF8040031280CD121480B
S31501A0757000682349884207D101A8009001231E4A29
S31501A0758001212220FAF78BFF9DF8040016BD1CB538
S31501A0759000208DF8040000200400E4B2092C26D2B4
S31501A075A01448007A000280B21249497A0843134965
S31501A075B0E4B231F81410884217D10E4880881149D7
S31501A075C0E4B2095D89B288420BD013208DF804007C
S31501A075D001A800900123084A01212220FAF75FFFA2
S31501A075E002E000208DF8040001E0641CD5E79DF8B7
S31501A075F0040016BDEC3D000017F1DA188C3A000024
S31501A07600F117DA18803A0000030011E30400000A1A
S31501A07610012052E20130D1240130C024F9FFFF8AB2
S31501A076201EFF2FE1030010E31200001A102052E200
S31501A076300500003A30002DE93810B1E8102052E2D9
S31501A076403810A0E8FBFFFF2A3000BDE8823EB0E17A
S31501A076500810B1280810A0280430914404308044B1
S31501A07660822FB0E1B220D1200130D144B220C02076
S31501A076700130C0441EFF2FE1042052E21000003A5F
S31501A07680010010E30600001A043091E4042052E23E
S31501A07690B230C0E06338A0E1B230C0E0F9FFFF2A02
S31501A076A0070000EA043091E4042052E20130C0E46C
S31501A076B06334A0E1B230C0E06338A0E10130C0E498
S31501A076C0F7FFFF2A04208232012052E20130D124A1
S31501A076D00130C024FBFFFF8A1EFF2FE100B583B056
S31501A076E000208DF80400FBF7F4F8012812D17F20C1
S31501A076F08DF80400DFF804030068DFF8041388425C
S31501A077000BD101A800900123BE4A01212720FAF737
S31501A07710C6FE02E000208DF804009DF804000EBD0F
S31501A0772000B583B000208DF80400B44880880028F5
S31501A077300BD113208DF8040001A800900123B14AB2
S31501A0774001212720FAF7ABFE02E000208DF8040004
S31501A077509DF804000EBD00B583B000208DF804008D
S31501A07760A648007A10F07F00112812D1A34880887C
S31501A0777000280BD113208DF8040001A80090012345
S31501A07780A04A01212720FAF78AFE02E000208DF8FF
S31501A0779004009A48007A10F07F00122812D1974867
S31501A077A0808805280BD213208DF8040001A800902B
S31501A077B00123944A01212720FAF771FE02E0002055
S31501A077C08DF804009DF804000EBD00B583B000201D
S31501A077D08DF804008948007A10F07F00112805D0A1
S31501A077E08648007A10F07F00122803D100208DF878
S31501A077F004000FE012208DF804008048006880493B
S31501A07800884207D101A8009001237E4A01212720A1
S31501A07810FAF745FE9DF804000EBD00B583B0002021
S31501A078208DF8040000208DF804007448007A10F049
S31501A078307F00112805D07148007A10F07F00122828
S31501A0784014D1FBF746F8022834D07E208DF8040027
S31501A078506A4800686A4988422CD101A80090012390
S31501A07860684A01212720FAF71AFE23E06348007A25
S31501A0787010F07F00012805D06048007A10F07F0043
S31501A07880022814D1FBF725F8012813D17E208DF803
S31501A0789004005A4800685A4988420BD101A80090B1
S31501A078A00123584A01212720FAF7F9FD02E0002019
S31501A078B08DF804009DF804000EBD00B583B000202C
S31501A078C08DF804004D48007A10F07F00112812D1DE
S31501A078D04A48808801280BD013208DF8040001A8FE
S31501A078E000900123474A01212720FAF7D8FD02E09B
S31501A078F000208DF804004148007A10F07F0012287C
S31501A0790012D13E48808805280BD013208DF804009B
S31501A0791001A8009001233B4A01212720FAF7BFFDC8
S31501A0792002E000208DF804009DF804000EBD00B50C
S31501A0793083B000208DF804003048007A10F07F0053
S31501A07940122813D130480078012803D100208DF8E0
S31501A0795004000EE024208DF8040001A80090012364
S31501A07960284A01212720FAF79AFD02E000208DF886
S31501A0797004009DF804000EBD00B583B000208DF86B
S31501A0798004002148407801280BD137208DF8040046
S31501A0799001A8009001231B4A01212720FAF77FFDA8
S31501A079A002E000208DF804009DF804000EBD00B58C
S31501A079B083B000208DF8040036208DF8040001A8BC
S31501A079C0009001230F4A01212720FAF768FD9DF8AF
S31501A079D004000EBD00B583B000208DF8040035204B
S31501A079E08DF8040001A800900123064A0121272051
S31501A079F0FAF755FD9DF804000EBD0000EC3D000010
S31501A07A00F117DA1817F1DA18F03E000000B583B0C5
S31501A07A1000208DF80400FAF75CFF032813D07F201D
S31501A07A208DF80400DFF8B4030068DFF8B4138842C8
S31501A07A300CD101A800900123DFF8A8230121282059
S31501A07A40FAF72DFD02E000208DF804009DF8040050
S31501A07A500EBD00B583B000208DF80400DFF87C03CD
S31501A07A60808802280CD213208DF8040001A800906A
S31501A07A700123DFF8702301212820FAF710FD02E087
S31501A07A8000208DF804009DF804000EBD00B583B05A
S31501A07A9000208DF80400DFF84403407A01281AD0AB
S31501A07AA0DFF83803407A022815D0DFF83003407A90
S31501A07AB0032810D031208DF80400C8480068C849B1
S31501A07AC088420BD101A800900123C64A0121282092
S31501A07AD0FAF7E5FC02E000208DF804009DF8040009
S31501A07AE00EBD00B583B000208DF80400BB48808888
S31501A07AF002280BD013208DF8040001A800900123C1
S31501A07B00B84A01212820FAF7CAFC02E000208DF824
S31501A07B1004009DF804000EBD00B583B000208DF8C9
S31501A07B200400FAF70BFF06280BD322208DF80400D8
S31501A07B3001A800900123AB4A01212820FAF7AFFC46
S31501A07B4013E0FAF7FFFEB0F5C87F0BD922208DF816
S31501A07B50040001A800900123A24A01212820FAF7D6
S31501A07B609EFC02E000208DF804009DF804000EBDE5
S31501A07B7000B583B000208DF804009848007A10F073
S31501A07B807F00002812D19548808802280BD21320A5
S31501A07B908DF8040001A800900123924A0121282012
S31501A07BA0FAF77DFC02E000208DF804008B48007AEC
S31501A07BB010F07F00012812D18848808802280BD2B4
S31501A07BC013208DF8040001A800900123854A012104
S31501A07BD02820FAF764FC02E000208DF804007F4813
S31501A07BE0007A10F07F00022812D17C4880880228F2
S31501A07BF00BD213208DF8040001A800900123794A25
S31501A07C0001212820FAF74BFC02E000208DF80400A0
S31501A07C107248007A10F07F00032812D16F4880883D
S31501A07C2002280BD213208DF8040001A8009001238D
S31501A07C306C4A01212820FAF732FC02E000208DF8D7
S31501A07C4004009DF804000EBD00B583B000208DF898
S31501A07C5004006248007A10F07F00002811D05F4826
S31501A07C60007A10F07F0001280BD05C48007A10F052
S31501A07C707F00032805D05948007A10F07F0002281A
S31501A07C8003D100208DF804000FE012208DF8040026
S31501A07C90524800685249884207D101A800900123A1
S31501A07CA0504A01212820FAF7FAFB9DF804000EBDDF
S31501A07CB000B583B000208DF804004848407A012819
S31501A07CC018D04648407A022814D04448407A03285E
S31501A07CD010D031208DF80400404800684049884200
S31501A07CE00BD101A8009001233E4A01212820FAF7D1
S31501A07CF0D6FB02E000208DF804009DF804000EBD1D
S31501A07D0000B583B000208DF804003448007A10F045
S31501A07D107F00002812D13148808802280BD0132079
S31501A07D208DF8040001A8009001232E4A01212820E4
S31501A07D30FAF7B5FB02E000208DF804002748007A87
S31501A07D4010F07F00012812D12448808802280BD088
S31501A07D5013208DF8040001A800900123214A0121D6
S31501A07D602820FAF79CFB02E000208DF804001B48AE
S31501A07D70007A10F07F00022812D1184880880228C4
S31501A07D800BD013208DF8040001A800900123154AF9
S31501A07D9001212820FAF783FB02E000208DF80400D8
S31501A07DA00E48007A10F07F00032812D10B48808874
S31501A07DB002280BD013208DF8040001A800900123FE
S31501A07DC0084A01212820FAF76AFB02E000208DF873
S31501A07DD004009DF804000EBD00000000EC3D00006B
S31501A07DE0F117DA1817F1DA1800B583B000208DF86B
S31501A07DF00400FAF76EFD022810D07F208DF804004A
S31501A07E0056480068564988420BD101A80090012323
S31501A07E10544A01212E20FAF742FB02E000208DF8F8
S31501A07E2004009DF804000EBD00B583B000208DF8B6
S31501A07E300400FAF78BFD012803D100208DF8040078
S31501A07E400AE033208DF8040001A800900123454AD9
S31501A07E5001212E20FAF723FB9DF804000EBD00B5E3
S31501A07E6083B000208DF804003C48808802280BD2FC
S31501A07E7013208DF8040001A800900123394A01219D
S31501A07E802E20FAF70CFB02E000208DF804009DF8E5
S31501A07E9004000EBD1CB531208DF80400002004009D
S31501A07EA0E4B2022C12D22D48007A000280B22B49EC
S31501A07EB0497A08432C49E4B231F81410884203D117
S31501A07EC000208DF8040001E0641CE9E79DF8040098
S31501A07ED031280CD1214800682149884207D101A83F
S31501A07EE0009001231F4A01212E20FAF7D8FA9DF806
S31501A07EF0040016BD1CB500208DF804000020040066
S31501A07F00E4B2022C26D21548007A000280B21349A7
S31501A07F10497A08431449E4B231F81410884217D1BA
S31501A07F200E4880881149E4B2095D89B288420BD016
S31501A07F3013208DF8040001A800900123094A01210C
S31501A07F402E20FAF7ACFA02E000208DF8040001E039
S31501A07F50641CD5E79DF8040016BD0000EC3D0000A9
S31501A07F60F117DA1817F1DA18A43A0000A83A0000B6
S31501A07F7000B583B000208DF80400FAF7AAFC012809
S31501A07F8010D17F208DF804007B4800687B49884288
S31501A07F900BD101A800900123794A01213120FAF7DA
S31501A07FA07EFA02E000208DF804009DF804000EBDC3
S31501A07FB000B583B000208DF80400FAF7C7FC0128AC
S31501A07FC003D100208DF804000AE033208DF80400C7
S31501A07FD001A8009001236A4A01213120FAF75FFA2C
S31501A07FE09DF804000EBD00B583B000208DF80400F5
S31501A07FF06148808803280BD213208DF8040001A8BC
S31501A08000009001235E4A01213120FAF748FA02E0E5
S31501A0801000208DF804009DF804000EBD1CB50020BB
S31501A080208DF804005448407A5349897A51EA0020D0
S31501A080300400A4B240F20220844219D0A4B2B4F53D
S31501A080407F4F15D0A4B24FF60170844210D03120D3
S31501A080508DF8040048480068484988420BD101A818
S31501A0806000900123464A01213120FAF718FA02E0CD
S31501A0807000208DF804009DF8040016BD1CB5002053
S31501A080808DF8040000208DF804003B48407A3A4957
S31501A08090897A51EA00200400A4B2200040F202210C
S31501A080A0401A06D04FF6FE41401A12D0401E20D0EB
S31501A080B02FE03148808807280AD013208DF80400C4
S31501A080C001A8009001232E4A01213120FAF7E7F9F0
S31501A080D02FE0294880880C280AD013208DF80400A7
S31501A080E001A800900123264A01213120FAF7D7F9E8
S31501A080F01FE02148808803280AD013208DF80400A8
S31501A0810001A8009001231E4A01213120FAF7C7F9DF
S31501A081100FE031208DF804001748006817498842FE
S31501A0812007D101A800900123154A01213120FAF7B0
S31501A08130B6F99DF8040016BD00B583B000208DF8F0
S31501A0814004000D48007A012803D100208DF804000F
S31501A081500FE012208DF804000748006807498842FD
S31501A0816007D101A800900123054A01213120FAF780
S31501A0817096F99DF804000EBDEC3D0000F117DA1842
S31501A0818017F1DA1800B583B000208DF804004A482B
S31501A08190808800280BD113208DF8040001A8009037
S31501A081A00123464A01213E20FAF779F902E000208F
S31501A081B08DF804009DF804000EBD00B583B0002023
S31501A081C08DF804003C48808801280BD013208DF837
S31501A081D0040001A800900123384A01213E20FAF7A4
S31501A081E05EF902E000208DF804009DF804000EBDA2
S31501A081F000B583B000208DF804002F48007A10F056
S31501A082007F00002812D12C48808800280BD113208A
S31501A082108DF8040001A800900123284A01213E20DF
S31501A08220FAF73DF902E000208DF804009DF804005C
S31501A082300EBD00B583B000208DF804001E48007A5B
S31501A0824010F07F00002803D100208DF804000FE074
S31501A0825012208DF80400184800681949884207D1F0
S31501A0826001A800900123154A01213E20FAF717F92A
S31501A082709DF804000EBD00B583B000208DF8040062
S31501A082800D48007A10F07F00002812D10A48808894
S31501A0829001280BD013208DF8040001A8009001231A
S31501A082A0064A01213E20FAF7FAF802E000208DF8ED
S31501A082B004009DF804000EBDEC3D000017F1DA188C
S31501A082C0F117DA1800B583B000208DF8040000205C
S31501A082D08DF80400FAF7FDFA022813D07F208DF855
S31501A082E00400DFF8A4040068DFF8A01488420CD1CA
S31501A082F001A800900123DFF8982401213420FAF780
S31501A08300CEF802E000208DF804009DF804000EBD11
S31501A0831000B583B000208DF80400FAF717FB0128F9
S31501A0832003D100208DF804000BE033208DF8040062
S31501A0833001A800900123DFF8582401213420FAF77F
S31501A08340AEF89DF804000EBD00B583B000208DF8EF
S31501A083500400DFF8340480880A280CD013208DF895
S31501A08360040001A800900123DFF824240121342070
S31501A08370FAF795F802E000208DF804009DF80400B4
S31501A083800EBD2DE9FC4700208DF8040000208DF8D4
S31501A0839004000020DFF8FC1308700020DFF8F813B2
S31501A083A00870DFF8F0034078012840F02B819DF892
S31501A083B00400002810D1DFF8D003007A00280BD0E2
S31501A083C031208DF8040001A800900123DFF8C02315
S31501A083D001213420FAF763F89DF80400002810D192
S31501A083E0DFF8A403407A44280BD031208DF804008D
S31501A083F001A800900123DFF8982301213420FAF780
S31501A084004EF89DF8040000281DD1DFF87C03437BBC
S31501A08410DFF87403027BDFF87003C17ADFF8680323
S31501A08420807AFAF7A2FE0400B4F1D17F0BD03120F5
S31501A084308DF8040001A800900123DFF8542301213F
S31501A084403420FAF72CF89DF8040000281DD1DFF896
S31501A084503803437CDFF83003027CDFF82C03C17BB1
S31501A08460DFF82403807BFAF780FE0500B5F5E81F47
S31501A084700BD331208DF8040001A800900123DFF869
S31501A08480102301213420FAF70AF89DF804000028E8
S31501A0849010D1DFF8F40280880A280BD013208DF8BA
S31501A084A0040001A800900123DFF8E4220121342071
S31501A084B0F9F7F5FF9DF80400002810D1DFF8DC02DA
S31501A084C0007801280BD070208DF8040001A8009037
S31501A084D00123DFF8BC2201213420F9F7E0FF9DF842
S31501A084E00400002840F04C810120DFF8AC1208738B
S31501A084F00120DFF8A4120870DFF89C02C0F80C5125
S31501A085000020DFF89412C1F81001DFF8940204608C
S31501A08510DFF88C0245600120DFF88812DFF87822A7
S31501A0852092F8142114235A438854DFF87802DFF80D
S31501A08530681291F81411142251430844DFF860120D
S31501A0854009684160DFF85802007910F0030F14D0D2
S31501A08550DFF85002DFF8401291F8141114225143AA
S31501A085600844DFF83C124968091DDFF83422127964
S31501A0857012F00302891A81600CE0DFF82802DFF805
S31501A08580181291F81411142251430844DFF810125D
S31501A0859049688160DFF80C02DFF8FC1191F814112B
S31501A085A0142251430844DFF8FC11DFF8EC2192F8BC
S31501A085B0142114235A4311444968DFF8E42152686F
S31501A085C05118C160DFF8D00190F81401401CDFF802
S31501A085D0C81181F814012020DFF8AC11087200201F
S31501A085E0DFF8A4114872E220DFF89C118872DFF847
S31501A085F0B80100900323DFF8982100213420F9F770
S31501A086004EFFBDE09DF80400002810D1DFF87801E7
S31501A08610007A00280BD031208DF8040001A8009023
S31501A086200123DFF86C2101213420F9F738FF9DF8E9
S31501A086300400002810D1DFF85001407A44280BD05D
S31501A0864031208DF8040001A800900123DFF8402114
S31501A0865001213420F9F723FF9DF8040000281ED13B
S31501A08660DFF82401437BDFF82001027BDFF8180144
S31501A08670C17ADFF81401807AFAF777FD0400DFF8F2
S31501A086802C0184420BD031208DF8040001A8009062
S31501A086900123DFF8FC2001213420F9F700FF9DF822
S31501A086A0040000281CD1DFF8E000437CDFF8D800E5
S31501A086B0027CDFF8D400C17BDFF8CC00807BFAF71F
S31501A086C054FD0500202D0BD031208DF8040001A802
S31501A086D000900123DFF8B82001213420F9F7DFFE4D
S31501A086E09DF80400002810D1DFF89C0080880A2894
S31501A086F00BD013208DF8040001A800900123DFF808
S31501A08700902001213420F9F7CAFE9DF80400002823
S31501A0871036D14FF48C760027DFF87C803A00310001
S31501A087204046FCF7A2EB4FF488785FF00009DFF82A
S31501A0873064A04A4641465046FCF796EB00201549EF
S31501A08740487014484460134885605FF0FF301149B2
S31501A08750C86001200F49087401200E490870202025
S31501A0876009490872002008494872E2200649887220
S31501A087700D4800900323064A00213420F9F78FFE05
S31501A087809DF80400BDE8F687EC3D0000F117DA1864
S31501A0879017F1DA18743F000084400000A6540000C7
S31501A087A0B0410000EC420000F43D000000009F0132
S31501A087B000B583B000208DF80400FAF78AF80228E4
S31501A087C013D07F208DF80400DFF89C000068DFF845
S31501A087D09C1088420CD101A800900123DFF89020BB
S31501A087E001213620F9F75BFE02E000208DF8040096
S31501A087F09DF804000EBD00B583B000208DF80400DD
S31501A08800DFF86400808802280BD213208DF80400BB
S31501A0881001A800900123164A01213620F9F73FFE4F
S31501A0882002E000208DF804009DF804000EBD1CB5E1
S31501A0883000208DF804000C488088401E0400A4B2D4
S31501A08840E12C0BDB13208DF8040001A80090012375
S31501A08850074A01213620F9F722FE02E000208DF811
S31501A0886004009DF8040016BDEC3D0000F117DA18CE
S31501A0887017F1DA1800B583B000208DF80400FAF7D5
S31501A0888028F8022811D07F208DF80400DFF85C00BB
S31501A088900068174988420BD101A800900123154A07
S31501A088A001213720F9F7FBFD02E000208DF8040035
S31501A088B09DF804000EBD00B583B000208DF804001C
S31501A088C00A48808800280BD013208DF8040001A83F
S31501A088D000900123074A01213720F9F7E0FD02E0C4
S31501A088E000208DF804009DF804000EBDEC3D0000AB
S31501A088F0F117DA1817F1DA1800B583B000208DF850
S31501A089000400F9F7E6FF032810D07F208DF80400B4
S31501A0891089480068894988420BD101A800900123A2
S31501A08920874A01218520F9F7BAFD02E000208DF8DA
S31501A0893004009DF804000EBD00B583B000208DF89B
S31501A0894004007D48808800280BD113208DF80400EF
S31501A0895001A8009001237A4A01218520F9F79FFDFC
S31501A0896002E000208DF804009DF804000EBD00B5BC
S31501A0897083B000208DF804006F48808801280BD0B1
S31501A0898013208DF8040001A8009001236C4A01214F
S31501A089908520F9F784FD02E000208DF804009DF8FA
S31501A089A004000EBD00B583B000208DF80400F9F7D0
S31501A089B0C5FF06280BD322208DF8040001A800903C
S31501A089C001235F4A01218520F9F769FD13E0F9F733
S31501A089D0B9FFB0F5C87F0BD922208DF8040001A8F4
S31501A089E000900123564A01218520F9F758FD02E09E
S31501A089F000208DF804009DF804000EBD00B583B0DB
S31501A08A0000208DF804004C48007A10F07F00012860
S31501A08A1012D14948808800280BD113208DF8040073
S31501A08A2001A800900123464A01218520F9F737FDC7
S31501A08A3002E000208DF804003F48007A10F07F0084
S31501A08A40022812D13C48808800280BD113208DF82A
S31501A08A50040001A800900123394A01218520F9F7D4
S31501A08A601EFD02E000208DF804009DF804000EBD55
S31501A08A7000B583B000208DF804002F48007A10F0CD
S31501A08A807F00012805D02C48007A10F07F0002282B
S31501A08A9003D100208DF804000FE012208DF8040008
S31501A08AA0254800682549884207D101A800900123DD
S31501A08AB0234A01218520F9F7F2FC9DF804000EBD99
S31501A08AC000B583B000208DF804001B48007A10F091
S31501A08AD07F00012812D11848808801280BD01320C5
S31501A08AE08DF8040001A800900123154A01218520D3
S31501A08AF0F9F7D5FC02E000208DF804000E48007AB3
S31501A08B0010F07F00022812D10B48808801280BD0D3
S31501A08B1013208DF8040001A800900123084A012121
S31501A08B208520F9F7BCFC02E000208DF804009DF831
S31501A08B3004000EBD00000000EC3D0000F117DA189C
S31501A08B4017F1DA1880B5FCF789FD364908800120AE
S31501A08B503449887000203349C87000203149087112
S31501A08B6000203049487100202E49887100202D49E6
S31501A08B70C87100F0F3FB01BD10B52A488078002822
S31501A08B8047D000F00FFCFCF769FD04002000254941
S31501A08B90098880B2884244D02248048000F008FCAB
S31501A08BA020480079401C1F4908711E4800790528F4
S31501A08BB004D300201B49087100F0FEFB1948407937
S31501A08BC0401C18494871174840790A2804D3002047
S31501A08BD01449487100F0F6FB12488079401C1149EE
S31501A08BE0887110488079192804D300200D4988710D
S31501A08BF0C046C0460B48C079401C0A49C8710948FD
S31501A08C00C07932280DD300200649C871C046C04696
S31501A08C1007E0C046C04603488078002801D1FCF78A
S31501A08C20BBFF10BDD43D000080B500F0CFFB01BD58
S31501A08C3080B5C046C04601BD2DE9F04782460C006D
S31501A08C4000F020F90500002D01D106205AE050467A
S31501A08C5000F070F900280AD11AF1807000F06AF9C3
S31501A08C60012802D11AF1807A01E004204AE01AF023
S31501A08C70030F01D0042045E00021504600F065F91C
S31501A08C8007000121504600F060F9804600205028D7
S31501A08C9002DA00BF401CFAE7AA203860002050285B
S31501A08CA002DA00BF401CFAE75520C8F800000020F0
S31501A08CB0502802DA00BF401CFAE780203860002065
S31501A08CC0502802DA00BF401CFAE7AA20386000202B
S31501A08CD0502802DA00BF401CFAE75520C8F8000068
S31501A08CE03020CAF80000002C08D00020814659F097
S31501A08CF00809484600F0D9F8060001E00020060060
S31501A08D003000C0B2BDE8F0872DE9F84F04000D0090
S31501A08D10160000F0B7F800900098002801D10620AF
S31501A08D205EE0200000F006F900280AD114F1807057
S31501A08D3000F000F9012802D114F1807401E00420A9
S31501A08D404EE014F0030F01D0042049E000212000D9
S31501A08D5000F0FBF880460121200000F0F6F88146DC
S31501A08D60002083461FFA8BFBBBF1370F05D200BF4C
S31501A08D70FEF70AF91BF1010BF4E7AA20C8F80000D7
S31501A08D805520C9F80000A020C8F80000002083469D
S31501A08D901FFA8BFBBBF1370F05D200BFFEF7F4F824
S31501A08DA01BF1010BF4E72560002083461FFA8BFB1C
S31501A08DB0BBF1370F05D200BFFEF7E6F81BF1010B99
S31501A08DC0F4E7002E08D0002082465AF0400A504609
S31501A08DD000F06BF8070001E0002007003800C0B2E0
S31501A08DE0BDE8F28F2DE9F84304000D0000F04AF822
S31501A08DF00600002E01D1062028E0200000F09AF8F6
S31501A08E0000280AD114F1807000F094F8012802D14B
S31501A08E1014F1807401E0042018E014F0030F01D0CE
S31501A08E20042013E020688046002D0BD00020814647
S31501A08E3059F04009484600F038F80700FFB2002F64
S31501A08E4004D101E0404601E04046FFE7BDE8F283D8
S31501A08E5038B500F051FB002801D1032011E000F044
S31501A08E6011F80500002D01D106200AE000F0D4F882
S31501A08E7001206C49087000F093F80400E007FAD4C9
S31501A08E80002032BD38B5012467480078C0B2002859
S31501A08E9002D10020040006E000F082F80500E807F0
S31501A08EA001D400200400200032BD70B504000025C5
S31501A08EB000F076F80600344203D0C6F3400000283D
S31501A08EC0F6D0C6F34000002803D0FFF7C1FF01206A
S31501A08ED005002800C0B270BD01005448814204D3E8
S31501A08EE0B1F1D07F01D2012000E00020704701003E
S31501A08EF0B1F1D07F04D3B1F1E07F01D2012000E02E
S31501A08F000020704710B504002000FFF7F0FF0028ED
S31501A08F1001D001200DE02000FFF7DEFF002807D0D9
S31501A08F204248844204D3B4F1D07F01D2012000E0AB
S31501A08F30002010BD10B504002000FFF7E3FF0128B3
S31501A08F4001D1012000E0002010BD70B504000D0084
S31501A08F5000262000FFF7C0FF01280BD1EDB2002D9E
S31501A08F6002D140F6A82001E040F25450610B49031A
S31501A08F70461813E02000FFF7C5FF01280BD1EDB27B
S31501A08F80002D02D140F6A82001E040F25450210C58
S31501A08F900904461802E07FF00F000600300070BDFC
S31501A08FA0234909680800704738B5002400F0A4FADF
S31501A08FB0002802D10320040013E0F8F760E80500B9
S31501A08FC072B61C480078C0B2012802D0062004005F
S31501A08FD004E000F021F80120134908702800F8F7F1
S31501A08FE052E82000C0B232BD38B5002400F084FAA0
S31501A08FF0002802D1032004000BE0F8F740E80500A1
S31501A0900072B600F009F80020074908702800F8F7A1
S31501A090103AE82000C0B232BD074808490860704747
S31501A0902000000000468018B1448018B100009F01DD
S31501A09030381041B0580319B1A5F161CF001041B064
S31501A090400020B0E3330100EA2DE9F04F83B004001C
S31501A0905000F052FA01900198002801D10320D7E02F
S31501A09060002C01D10420D3E000F0D4F8009011EE39
S31501A09070100F0700BFF34F8F7F087F0001EE107F0F
S31501A09080BFF36F8F10EE900F050000200600C5F309
S31501A090900720864280F0A0801C2000FB06F0204419
S31501A090A08068012840F08B8006EE126F1C2000FB21
S31501A090B006F02044806906EE110F16EE510F824686
S31501A090C01C2000FB06F02044007F60F3450A5AF0FD
S31501A090D0010A0020804600208146B9F1080F0CD272
S31501A090E01C2000FB06F020444844407B10FA09F0FE
S31501A090F050EA080819F10109EFE75FFA88F868F361
S31501A091000F2A06EE51AF16EE910F83461C2000FBE7
S31501A0911006F02044007B60F30A2B1C2000FB06F01E
S31501A091202044407F60F3000B1C2000FB06F0204486
S31501A09130407FC0B24008C0B260F3410B1C2000FBC7
S31501A0914006F02044407FC0F38200C0B260F3C50B95
S31501A091501C2000FB06F02044807F60F3820B1C20BC
S31501A0916000FB06F02044407D60F30C3B1C2000FB75
S31501A0917006F02044407F10281ED11C2000FB06F0DB
S31501A091802044C07F60F3000B1C2000FB06F02044A6
S31501A09190C07FC0B24008C0B260F3410B3BF03800BB
S31501A091A01C2101FB06F1214491F820105BEAC101C3
S31501A091B011F0380151EA000B06EE91BF0AE006EE66
S31501A091C0126F16EE510F82465FEA5A0A5FEA4A0A01
S31501A091D006EE51AF761C5AE72068012814D111EE8C
S31501A091E0100F0700BFF34F8F57F0010760680128E2
S31501A091F001D1012000E0002060F3514701EE107F6C
S31501A09200BFF34F8FBFF36F8F009800F055F8002082
S31501A09210BDE8FE8F2DE9F05F11EE101F41F20402A9
S31501A0922011EA020045D001B411EE101F21F48051BC
S31501A0923021F00401BFF34F8F01EE101FBFF36F8F13
S31501A0924030EE300F10F0E0634FEAD35330D04FF039
S31501A09250000A0AEB5A0220FA02F101F0070123D013
S31501A0926040EE10AFBFF36F8F30EE101F01F0070273
S31501A0927002F1040240F2FF3414EAD104B4FA84F5EF
S31501A0928047F6FF7717EA5137A14609FA05F64AEAE2
S31501A09290060B07FA02F84BEA080B07EE5ABFB9F11B
S31501A092A00109F2DA7F1EEFDA0AF1020A5345D0DC90
S31501A092B001BCBDE8F05F704711EE101F41EA000145
S31501A092C0BFF34F8F0FEE150F07EE150F01EE101F0F
S31501A092D0BFF36F8F7047000030B4C0B2002802D12F
S31501A092E00124230001E06B242300C9B2002901D087
S31501A092F053F00403D2B2002A01D053F010035FF059
S31501A09300FF34064D2C60064C237030BC70470549CE
S31501A09310086070470449096808007047048071B461
S31501A09320008071B4088071B40C8071B480B500F06E
S31501A093300FF9F7F7B3FE00F093F900F0E6F9FCF7A1
S31501A093405FFA00F066FA00F047F800F0B1F8FCF712
S31501A0935061FD002801D100F0CFFA01BD10B5FDF7DE
S31501A09360D9FDFDF755F8F9F72AFC04000A4884420D
S31501A0937005D00A48844202D00948844201D1FDF7AA
S31501A0938027F8F7F76EF9FCF749F9F7F7ABFE61B6DF
S31501A0939062B6F9F739FA10BD633658853663855832
S31501A093A0A35A7AA780B5F7F747FFF8F7EBFE01BDF9
S31501A093B080B5FCF7F7FD01BD80B5F9F700FBF7F71E
S31501A093C0DBFD01BD80B5FCF707FE01BD80B53220EE
S31501A093D0F7F73CFF01BD000070B410EE905F2900C5
S31501A093E000252C00C1F30725AC424FD22F4D2601F3
S31501A093F0AD59012D3FD106EE124F2C4D2601354414
S31501A09400AD6806EE115F16EE515F2A00274D2601C3
S31501A0941035442D7B65F3450252F0010232F47F42B9
S31501A0942006EE512F16EE915F2B00032565F30A2355
S31501A094301E4D260135446D7B65F300031B4D2601A8
S31501A0944035446D7B6D0865F34103184D26013544FE
S31501A094506D7BAD0865F3C503144D26013544AD7B7F
S31501A0946065F38203114D260135442D7965F30C333D
S31501A0947006EE913F08E006EE124F16EE515F2A0066
S31501A094805208520006EE512F641CABE711EE105F95
S31501A094902800BFF34F8F50F0010050F4003001EEC9
S31501A094A0100FBFF36F8F70BC70470000C4A1A0015D
S31501A094B011EE301F080030F0380040F4804050F023
S31501A094C0100001EE300F11EE101F080050F480506D
S31501A094D0002107EE151F01EE100FBFF36F8F11EEDE
S31501A094E0101F080050F00400BFF34F8F00210FEEAC
S31501A094F0151F01EE100F704780B500F006F8102871
S31501A0950001D0012000E0002002BDEFF30081080098
S31501A0951010F01F007047000004402DE90230A0E1C1
S31501A0952002E0A0E102C0A0E1101051E20C50A02877
S31501A09530FCFFFF8A81CEB0E10C00A0280420804464
S31501A09540811FB0E1B220C0200120C0440480BDE843
S31501A095503748384908600FF23100374908600FF2E1
S31501A095605800364908600FF2810035490860354830
S31501A09570354908603548006850F480703349086061
S31501A0958033482C490860704700BFFDE710402DE91C
S31501A095900040B0E1B8009FE5000090E5000050E36F
S31501A095A00300000A0400B0E1A4109FE5001091E5B4
S31501A095B031FF2FE11080BDE8FF5F2DE90D10A0E17D
S31501A095C000004FE1200010E3B2005E11FF0CC013B2
S31501A095D004001E05FF04C003EBFFFFEBFF5FBDE820
S31501A095E00EF0B0E11EFF2FE183B015EE300F029011
S31501A095F015EE310F019016EE500F009003B0704793
S31501A0960083B015EE100F029015EE110F019016EE14
S31501A09610100F009010480068C0F38010002805D0F4
S31501A096200E48006850F040000C49086003B070472E
S31501A0963007B0C5AC58FFFEFF84FFFEFF88FFFEFF03
S31501A096408CFFFEFF3CA7A00190FFFEFF60FFFEFF7F
S31501A09650F6EC07B078A7A0012C1010B0301010B00E
S31501A0966079487A49086001207949096860F30101BE
S31501A0967077480160744875490860002075490870EB
S31501A0968075487649086005207549096860F30301A4
S31501A096907348016073487449086074480078C0B281
S31501A096A00128FAD07248006830F04070704908600D
S31501A096B070486D4908606D480078C0B20028FAD09C
S31501A096C06D486E4908606E480068C0F30020002806
S31501A096D0F9D16B48006830F0407069490860684864
S31501A096E0006830F440306649086066480068400862
S31501A096F040006449086064486049086060480068A1
S31501A09700C0F300200028F9D070471CB4002319002B
S31501A0971000231A000023180000238DF8043000232B
S31501A097208DF8003051F0407151F4700151F470215F
S31501A09730012363F31D72032363F30F32032363F340
S31501A097400B2252F07F0250F001009DF8043013F075
S31501A097507F038DF804309DF8003013F07F038DF858
S31501A0976000309DF8003053F010038DF80030474BC0
S31501A097701B6833F0C053454C23600123444C23702E
S31501A09780444B1B68D3F50033DB095B1E63F30F0162
S31501A0979052F04062404B414C23603E4B1B6813F193
S31501A097A080633F4C23603F4B19603F4B1A603F4B90
S31501A097B018609DF804303E4C23709DF800303D4C56
S31501A097C0237001233C4C237001233C4C237040F2AF
S31501A097D03F3363F30F0152F040622F4B384C2360A5
S31501A097E0384B394C2360394B1960394B1A60394BC8
S31501A097F018609DF80430384C23709DF80030374C22
S31501A0980023700123364C23700123364C237013BCDD
S31501A09810704735480078C0B20028FAD00020264902
S31501A09820087001203149087031480078C0B200287B
S31501A09830FAD000202A49087001202E49087000207C
S31501A098401249086070470000A5F161CF001041B030
S31501A09850081041B0808018B1A5F16DCF002041B0AC
S31501A09860082041B0CC5EC5AC080041B0080018B1D3
S31501A09870000041B00CB1CC5E1F55CC5E0C8010B07F
S31501A09880008010B0188010B00CB11F55001070B434
S31501A098901F8000B78CA1A00170A4A005080070B418
S31501A098A00C0070B4000070B4040070B4100070B461
S31501A098B0150070B4170070B41F0000B71D0000B7E3
S31501A098C0480070B4006000024C0070B4400070B44F
S31501A098D0440070B4500070B4550070B4570070B411
S31501A098E01F0200B71D0200B73F0000B7800000B7F6
S31501A098F03F0200B7800200B738B50020DFF8FC10A0
S31501A0990008600120DFF8F8100870DFF8F800007889
S31501A09910C0B20028F9D00020DFF8E41008704FF497
S31501A09920FA60ADF8000001208DF8020001208DF843
S31501A099300300AD09AD0135F47C5535F4F81568463B
S31501A0994000F026F80400DFF8BC000078C0B20028B9
S31501A09950F9D1DFF8B4000480DFF8B0000560DFF8C4
S31501A09960B000006830F03000DFF8A4100860DFF81E
S31501A09970A400DFF8A41008607F20DFF8A01008601B
S31501A099800120DFF89C10087001201D49087031BD27
S31501A099902DE9F04104000020804620880700B7F594
S31501A099A0F067BFB240F26D1000FB07F010FA88F81D
S31501A099B0BFB2F81C800810FA88F8208800F034F8A5
S31501A099C00600012005002800A178C0B288420DD268
S31501A099D01448F6B20C2101FB06F10844EDB2284465
S31501A099E010F8010C58FA80F86D1CECE7E078401EDF
S31501A099F010EB0808404680B2BDE8F0810C8061B04A
S31501A09A0000008CB020008CB01C8061B0188061B0C1
S31501A09A10008061B009851E00148061B0108061B01C
S31501A09A2080018CB024A7A00101000322114202D01B
S31501A09A300022100001E001221000C0B27047000010
S31501A09A4000000000963007772C610EEEBA510999F5
S31501A09A5019C46D078FF46A7035A563E9A395649E51
S31501A09A603288DB0EA4B8DC791EE9D5E088D9D29775
S31501A09A702B4CB609BD7CB17E072DB8E7911DBF90D1
S31501A09A806410B71DF220B06A4871B9F3DE41BE84F5
S31501A09A907DD4DA1AEBE4DD6D51B5D4F4C785D38351
S31501A09AA056986C13C0A86B647AF962FDECC9658AF5
S31501A09AB04F5C0114D96C0663633D0FFAF50D088D51
S31501A09AC0C8206E3B5E10694CE44160D5727167A2F5
S31501A09AD0D1E4033C47D4044BFD850DD26BB50AA551
S31501A09AE0FAA8B5356C98B242D6C9BBDB40F9BCAC75
S31501A09AF0E36CD832755CDF45CF0DD6DC593DD1ABD1
S31501A09B00AC30D9263A00DE518051D7C81661D0BFF4
S31501A09B10B5F4B42123C4B3569995BACF0FA5BDB850
S31501A09B209EB802280888055FB2D90CC624E90BB1F4
S31501A09B30877C6F2F114C6858AB1D61C13D2D66B650
S31501A09B409041DC760671DB01BC20D2982A10D5EFB4
S31501A09B508985B1711FB5B606A5E4BF9F33D4B8E810
S31501A09B60A2C9077834F9000F8EA8099618980EE1B4
S31501A09B70BB0D6A7F2D3D6D08976C6491015C63E610
S31501A09B80F4516B6B62616C1CD83065854E0062F234
S31501A09B90ED95066C7BA5011BC1F4088257C40FF590
S31501A09BA0C6D9B06550E9B712EAB8BE8B7C88B9FCB4
S31501A09BB0DF1DDD62492DDA15F37CD38C654CD4FB10
S31501A09BC05861B24DCE51B53A7400BCA3E230BBD4B4
S31501A09BD041A5DF4AD795D83D6DC4D1A4FBF4D6D310
S31501A09BE06AE96943FCD96E34468867ADD0B860DAB4
S31501A09BF0732D0444E51D03335F4C0AAAC97C0DDD10
S31501A09C003C710550AA41022710100BBE86200CC933
S31501A09C1025B56857B3856F2009D466B99FE461CE8F
S31501A09C200EF9DE5E98C9D9292298D0B0B4A8D7C7B3
S31501A09C30173DB359810DB42E3B5CBDB7AD6CBAC00F
S31501A09C402083B8EDB6B3BF9A0CE2B6039AD2B1742B
S31501A09C503947D5EAAF77D29D1526DB048316DC7387
S31501A09C60120B63E3843B64943E6A6D0DA85A6A7A2B
S31501A09C700BCF0EE49DFF099327AE000AB19E077D87
S31501A09C8044930FF0D2A3088768F2011EFEC20669AB
S31501A09C905D5762F7CB67658071366C19E7066B6E07
S31501A09CA0761BD4FEE02BD3895A7ADA10CC4ADD672B
S31501A09CB06FDFB9F9F9EFBE8E43BEB717D58EB06087
S31501A09CC0E8A3D6D67E93D1A1C4C2D83852F2DF4F2B
S31501A09CD0F167BBD16757BCA6DD06B53F4B36B24887
S31501A09CE0DA2B0DD84C1B0AAFF64A0336607A04412B
S31501A09CF0C3EF60DF55DF67A8EF8E6E3179BE694687
S31501A09D008CB361CB1A8366BCA0D26F2536E26852AA
S31501A09D1095770CCC03470BBBB91602222F26055506
S31501A09D20BE3BBAC5280BBDB2925AB42B046AB35C2A
S31501A09D30A7FFD7C231CFD0B58B9ED92C1DAEDE5B86
S31501A09D40B0C2649B26F263EC9CA36A750A936D026A
S31501A09D50A906099C3F360EEB8567077213570005C6
S31501A09D60824ABF95147AB8E2AE2BB17B381BB60CEA
S31501A09D709B8ED2920DBED5E5B7EFDC7C21DFDB0B46
S31501A09D80D4D2D38642E2D4F1F8B3DD686E83DA1F6A
S31501A09D90CD16BE815B26B9F6E177B06F7747B718C6
S31501A09DA0E65A0888706A0FFFCA3B06665C0B01116A
S31501A09DB0FF9E658F69AE62F8D3FF6B6145CF6C16C6
S31501A09DC078E20AA0EED20DD75483044EC2B303396A
S31501A09DD0612667A7F71660D04D476949DB776E3EC6
S31501A09DE04A6AD1AEDC5AD6D9660BDF40F03BD837EA
S31501A09DF053AEBCA9C59EBBDE7FCFB247E9FFB53046
S31501A09E001CF2BDBD8AC2BACA3093B353A6A3B42469
S31501A09E100536D0BA9306D7CD2957DE54BF67D923C5
S31501A09E202E7A66B3B84A61C4021B685D942B6F2A69
S31501A09E3037BE0BB4A18E0CC31BDF055A8DEF022DC5
S31501A09E400000E00020000100E60020000200E6007C
S31501A09E5020000300E00020000400E000200005002F
S31501A09E60E00020000600E00020000700E00020003E
S31501A09E700800E00020000900E01020000A00E01020
S31501A09E8020000B00E01020000C00E01020000D00C7
S31501A09E90E00020000E00E00020000F00E0002000FE
S31501A09EA01000E00020001100E00020001200E010E8
S31501A09EB020001300C01020001400C01020001500BF
S31501A09EC0C01020001600E01020001700C0102000CE
S31501A09ED01800E00020001900C01000101A00E200CE
S31501A09EE022001B00C01020001C00C01020001D0075
S31501A09EF0E00020001E00E00020001F00E00020007E
S31501A09F002000C01000102100E00020002200E01077
S31501A09F1020102300C01020002400E01020102500EE
S31501A09F20E00020002600E01020102700C01000103D
S31501A09F302800E00020002900E00020002A00E0100F
S31501A09F4020102B00E60020002C00E00020002D00B0
S31501A09F50C01000102E00C01000102F00C01000105D
S31501A09F603000C01000103100C01020003200E50002
S31501A09F7020003300E50020003400E5002000350074
S31501A09F80E50020003600E50020003700E5002000AE
S31501A09F903800E50020003900E50020003A00C01095
S31501A09FA000103B00E01020003C00E01020003D0026
S31501A09FB0E01020003E00C10020003F00C1002000AB
S31501A09FC04000E01020004100C10020004200200016
S31501A09FD020004300E00020004400E00020004500EE
S31501A09FE0E50020004600E50020004700E50020002E
S31501A09FF04800E00020004900C10020004A00C1003D
S31501A0A00020004B00C00020004C00C10020004D00E4
S31501A0A010C00020004E00E00020004F00E00020001C
S31501A0A0205000E00020005100E00020005200E000B6
S31501A0A03020005300E00020005400E000200055005D
S31501A0A040E00020005600E00020005700E0002000BC
S31501A0A0505800E01020105900C01020005A00E0104E
S31501A0A06020005B00E60020005C00E00020005D000F
S31501A0A070C010200000010CF100000FE11F00C0E399
S31501A0A080110080E300F021E100D19FE51F00C0E3AC
S31501A0A090120080E300F021E1F4D09FE51F00C0E3A8
S31501A0A0A0170080E300F021E1ECD09FE51F00C0E39B
S31501A0A0B01B0080E300F021E1E0D09FE51F00C0E393
S31501A0A0C0130080E300F021E1C8D09FE51F00C0E3A3
S31501A0A0D01F0080E300F021E1ACD09FE5A8009FE539
S31501A0A0E000C0A0E3040040E200C080E50C0050E1FE
S31501A0A0F0FBFFFF1A88C09FE53CFF2FE188009FE583
S31501A0A10000C0A0E3040040E200C080E50C0050E1DD
S31501A0A110FBFFFF1A00000FE11F00C0E3110080E35F
S31501A0A12000F021E17CD09FE51F00C0E3120080E38F
S31501A0A13000F021E170D09FE51F00C0E3170080E386
S31501A0A14000F021E168D09FE51F00C0E31B0080E37A
S31501A0A15000F021E15CD09FE51F00C0E3130080E37E
S31501A0A16000F021E144D09FE51F00C0E31F0080E37A
S31501A0A17000F021E128D09FE508C09FE51CFF2FE153
S31501A0A180FEFFFFEA2D93A00140A6A00180000000DA
S31501A0A19028000000200000001800000010000000A8
S31501A0A1A00800000000200000002100000029000096
S31501A0A1B080290000002A0000802A0000802A0000D1
S31501A0A1C0803A00000100000000000000000000002D
S31501A0A1D0160300000100000000000000000080003E
S31501A0A1E016030000010000000000000000000001AD
S31501A0A1F0170300000100000000000000000000029B
S31501A0A200160300000100000000000000000080020B
S31501A0A2100F03000001000000000000000000000480
S31501A0A2201803000001000000000000000000000E5D
S31501A0A2301308000001000000000000000000200E2D
S31501A0A2401308000001000000000000000000300E0D
S31501A0A2501303000001000000000000000000800EB2
S31501A0A2600F080000010000000000000000000050DF
S31501A0A27014040100010000000000000000002050AD
S31501A0A2801400010001000000000000000000405081
S31501A0A2901400010001000000000000000000009071
S31501A0A2A01B0001000100000001000000000000B039
S31501A0A2B01B010000000000000000000000000000DB
S31501A0A2C0040000000000A0010080A0010000A1017F
S31501A0A2D00080A1010000A2010080A2010000A3014B
S31501A0A2E00080A3010000A4010080A4010000A50133
S31501A0A2F00080A5010000A6010080A6010000A7011B
S31501A0A3000080A7010000A8010080A8010000A90102
S31501A0A3100080A9010000AA010080AA010000AB01EA
S31501A0A3200080AB010000AC010080AC010000AD01D2
S31501A0A3300080AD010000AE010080AE010000AF01BA
S31501A0A3400080AF010000B0010080B0010000B101A2
S31501A0A3500080B1010000B2010080B2010000B3018A
S31501A0A3600080B3010000B4010080B4010000B50172
S31501A0A3700080B5010000B6010080B6010000B7015A
S31501A0A3800080B7010000B8010080B8010000B90142
S31501A0A3900080B9010000BA010080BA010000BB012A
S31501A0A3A00080BB010000BC010080BC010000BD0112
S31501A0A3B00080BD010000BE010080BE010000BF01FA
S31501A0A3C00080BF010100000002000000040000009F
S31501A0A3D0080000001000000020000000400000005E
S31501A0A3E0800000000001000000020000000400003F
S31501A0A3F0000800000010000000200000004000003E
S31501A0A400008000000000010000000200000004001E
S31501A0A410000008000000100000002000000040001D
S31501A0A42000008000000000010000000200000004FE
S31501A0A43000000008000000100000002000000040FD
S31501A0A4400000008010B450F8041B79B1026843687B
S31501A0A45002440830DC0744BFA9F10104E31852F80D
S31501A0A460044B091F43F8044BF9D1ECE710BC704724
S31501A0A4700000000000000000000000000000000035
S31501A0A4800000000000000000000000000000000025
S31501A0A4900000000000000000000000000000000015
S31501A0A4A00000000000000000000000000000000005
S31501A0A4B000000000000000000000000000000000F5
S31501A0A4C000000000000000000000000000000000E5
S31501A0A4D000000000000000000000000000000000D5
S31501A0A4E000000000000000000000000000000000C5
S31501A0A4F001001000B846000001001800F84600004F
S31501A0A500010014005847000001007400A84700008C
S31501A0A51001006401784900000100EC00084F000029
S31501A0A52001001400B85200000100280008530000E1
S31501A0A5300000000000000000000000000000000074
S31501A0A5400000000000000000000000000000000064
S31501A0A5500000000000000000000000000000000054
S31501A0A56001000000040000001000000040000000EF
S31501A0A57000010000000400000010000000400000DF
S31501A0A58000000100000004000000100000004000CF
S31501A0A59000000001000000040000001000000040BF
S31501A0A5A0FFE1FF25A0010026FFE1FF250000002411
S31501A0A5B0A31BFCC300000000A31B00C000000000F9
S31501A0A5C0FAFFFF180AC84708FAFFFF3A0000400041
S31501A0A5D000000000000000000000000000000000D4
S31501A0A5E010B540F2F601C0F200017944A1F10C01C7
S31501A0A5F040F2FC04C0F200047C44A4F10C0404E083
S31501A0A6000A68081D114488470146A142F8D110BD28
S31501A0A610020202020202020202000000000201027C
S31501A0A62080F186F187F189F193F198F199F1000012
S31501A0A6302707000098F199F11206320001000000E7
S31501A0A6400100A0E30100B0E3000050E30000000A0E
S31501A0A650E2FFFFFA0000A0E300F020E3020000FA07
S31501A0A660080000FA080000EBFDFFFFEA80B5FEF73F
S31501A0A67069FAF8F72BFAFEF77FFAFCF785FCFAE7F9
S31501A0A680DFF800F0A0A6A001FFF7FABF261000E3AD
S31501A0A690021040E31800A0E3563412EFFAFFFFEAD6
S31501A0A6A00070B0E10700B0E1F7FFFFEBFDFFFFEAA5
S31501A0A6B0500F11EEF00880E3500F01EE0100A0E368
S31501A0A6C0950F07EE4004A0E3100AE8EE8007A0E389
S31501A0A6D0100AE1EE1EFF2FE16DFDFFFF3000000025
S31501A0A6E030FFFFFF803A00000000000003000000D9
S31501A0A6F0300000000003000000300000000003004D
S31501A0A70000003000000000030000003074A7A00183
S31501A0A71064A7A00154A7A001ECA6A00160A5A00171
S31501A0A720C4A3A0011F1C1F1E1F1E1F1F1E1F1E1F0D
S31501A0A7301F1D1F1E1F1E1F1F1E1F1E1F04E04EE2F0
S31501A0A7400F502DE904009FE530FF2FE10F90FDE8A2
S31501A0A7500196A0010F000000000F000000000F00ED
S31501A0A7600000000FFF0000000000FF00FF00000036
S31501A0A77000000000FFFF00000000000074F715179D
S70501A0A07445
